:020000040000FA
:1000000002EF00F00F013F0E926E000E936E000E95
:10001000946E030E956E0F0E966E000E386F000EE6
:10002000396F000E3A6F000E3B6F000E3C6F806A16
:10003000816A826A836A846A896A8A6A8B6A8C6A3C
:100040008D6A00018B8C006A016A026A036A046A85
:10005000056A066A076A086A096A0A6A0B6A0C6A0C
:100060000D6A0E6A0F6A106A116A126A136A146ABC
:10007000156A166A176A186A196A1A6A1B6A1C6A6C
:100080001D6A1E6A1F6A206A216A226A236A256A1B
:10009000266A276A296A246A286A2A6A2B6A2C6ACD
:1000A0002D6A2E6A2F6A306A316A326A336A346A7C
:1000B000356A366A376A386A396A3A6A3C6A3B6A2C
:1000C0003D6A3E6A3F6A406A416A426A436A446ADC
:1000D000456A466A476A486A496A4A6A4B6A4C6A8C
:1000E0004D6A4E6A506A516A526A536A546A556A36
:1000F000566A576A586A596A5A6A6EEC37F06EEC5B
:1001000037F06EEC37F06EEC37F02EEC2BF0C00EC3
:100110008A6E8C9C8C9E8C8A8C9A2DEC2CF03F0ED7
:100120008A6E8C9C8C9E8C8A8C9A50EC2CF08B8ADC
:1001300031EC2BF096EC37F0000EAA6E000EA96E93
:10014000A69EA69CA68000000000A850116E000E7E
:10015000AA6E010EA96EA69EA69CA68000000000B5
:10016000A850126E000EAA6E020EA96EA69EA69C44
:10017000A68000000000A850136E000EAA6E030EA9
:10018000A96EA69EA69CA68000000000A850146E32
:10019000000EAA6E040EA96EA69EA69CA680000064
:1001A0000000A850156E000EAA6E050EA96EA69E40
:1001B000A69CA68000000000A850166E000EAA6E35
:1001C000060EA96EA69EA69CA68000000000A85060
:1001D000176E000EAA6E070EA96EA69EA69CA6809C
:1001E00000000000A850186E000EAA6E080EA96E3E
:1001F000A69EA69CA68000000000A850196E000EC6
:10020000AA6E090EA96EA69EA69CA68000000000FC
:10021000A8501A6E000EAA6E0A0EA96EA69EA69C83
:10022000A68000000000A8504C6E6DEC2CF0B2ECE3
:100230002DF01D504E6E4CA423EF01F083A223EF4E
:1002400001F049EC36F0B2EC2DF080B280B650EF00
:1002500001F0070E5A5CD8B431EF01F05A2A52EF80
:1002600001F05A6A3EB652EF01F01550380B406E5D
:10027000380E405CD8B441EF01F0080E402643EF41
:1002800001F0000E406E1550C70B156E4050151250
:100290004CB266EC36F06DEC2CF03E8652EF01F07D
:1002A0003E965A6A80B47CEF01F0070E595CD8B4D0
:1002B0005DEF01F0592A7EEF01F0596A3EB47EEFFE
:1002C00001F01550380B406E000E405CD8B46DEF55
:1002D00001F0080E405E6FEF01F0380E406E1550D1
:1002E000C70B156E405015124CB266EC36F06DEC33
:1002F0002CF03E847EEF01F03E94596A4CB444ECFD
:1003000036F080B29EEF01F0070E585CD8B48CEF47
:1003100001F0582AA0EF01F0586A3EB2A0EF01F0B8
:10032000040E415CD8B498EF01F0412A99EF01F036
:10033000416A50EC2CF03E82A0EF01F03E92586AE8
:10034000000E415CD8B4BBEF01F0010E415CD8B4A3
:10035000B0EF0BF0020E415CD8B4E6EF11F0030EE3
:10036000415CD8B421EF21F0040E415CD8B4CDEF4C
:1003700026F023EF01F028EC2BF0410E34EC2BF0AB
:10038000B80E4DEC2BF0700E66EC2BF0100E66ECF8
:100390002BF0100E66EC2BF0100E66EC2BF0000E1E
:1003A00066EC2BF08DEC46F0000E66EC2BF0CDECFD
:1003B00045F0000E66EC2BF0ADEC45F0000E66EC5F
:1003C0002BF0CDEC45F0000E66EC2BF00DEC46F07A
:1003D000000E66EC2BF0CDEC46F0000E66EC2BF038
:1003E000CDEC45F0000E66EC2BF08DEC46F0BDEC4C
:1003F00048F09DEC46F02BEC2BF0400E34EC2BF04B
:10040000B80E4DEC2BF0ADEC46F0000E66EC2BF088
:100410008DEC45F0000E66EC2BF0ADEC46F0000ED6
:1004200066EC2BF0BDEC46F0000E66EC2BF09DEC7C
:1004300046F0000E66EC2BF0082A210E085CD8B4BA
:1004400027EF02F0100E66EC2BF01CEF02F0086AAA
:10045000700E66EC2BF028EC2BF0400E34EC2BF0F9
:10046000BA0E4DEC2BF01DA852EF02F0BDEC48F097
:10047000BDEC48F0BDEC48F0BDEC48F0000E66EC79
:100480002BF0BDEC48F0000E66EC2BF0BDEC48F014
:10049000000E66EC2BF0BDEC48F0000E66EC2BF085
:1004A0007CEF02F01BA49EEF02F0FF0E66EC2BF037
:1004B000EDEC47F0FF0E66EC2BF0FDEC47F0FF0E85
:1004C00066EC2BF0FF0E66EC2BF0FF0E66EC2BF0CB
:1004D0003DEC48F0FF0E66EC2BF03DEC47F0FF0ED4
:1004E00066EC2BF0DDEC47F0FF0E66EC2BF03DECFC
:1004F00048F0FF0E66EC2BF0082A1A0E085CD8B400
:1005000087EF02F0000E66EC2BF07CEF02F0086A39
:100510002BEC2BF0400E34EC2BF0BA0E4DEC2BF004
:10052000082A070E085CD8B49BEF02F0000E66ECB8
:100530002BF090EF02F0086A25EF03F0FF0E66EC57
:100540002BF03DEC48F0FF0E66EC2BF03DEC47F055
:10055000FF0E66EC2BF0DDEC47F0FF0E66EC2BF0A7
:100560003DEC48F0FF0E66EC2BF0000E66EC2BF035
:10057000000E66EC2BF01BA2EEEF02F0FF0E66EC15
:100580002BF0FDEC47F0FF0E66EC2BF02DEC48F065
:10059000FF0E66EC2BF09DEC47F0FF0E66EC2BF0A7
:1005A0007DEC47F0FF0E66EC2BF0EDEC47F0FF0E14
:1005B00066EC2BF01DEC47F0FF0E66EC2BF02BECFD
:1005C0002BF0400E34EC2BF0BA0E4DEC2BF0CDECB2
:1005D00047F0FF0E66EC2BF025EF03F0FF0E66EC04
:1005E0002BF03DEC47F0FF0E66EC2BF0FDEC47F0F6
:1005F000FF0E66EC2BF00DEC48F0FF0E66EC2BF0D6
:100600009DEC48F0FF0E66EC2BF0082A0D0E085CFE
:10061000D8B410EF03F0000E66EC2BF005EF03F0FA
:10062000086A2BEC2BF0400E34EC2BF0BA0E4DEC9C
:100630002BF0082A070E085CD8B424EF03F0000E54
:1006400066EC2BF019EF03F0086A2BEC2BF0480E48
:1006500034EC2BF0BA0E4DEC2BF01DB847EF03F045
:100660001BA647EF03F0FF0E66EC2BF00DEC48F0F5
:10067000FF0E66EC2BF02DEC48F0FF0E66EC2BF035
:10068000FDEC47F0FF0E66EC2BF053EF03F0082A69
:10069000140E085CD8B452EF03F0000E66EC2BF099
:1006A00047EF03F0086A2BEC2BF05D0E34EC2BF0D7
:1006B000BA0E4DEC2BF01DB87AEF03F01BB07AEFB9
:1006C00003F0FF0E66EC2BF05DEC47F0FF0E66ECDE
:1006D0002BF0DDEC47F0FF0E66EC2BF00DEC48F054
:1006E000FF0E66EC2BF08DEC47F0FF0E66EC2BF066
:1006F00086EF03F0082A1A0E085CD8B485EF03F0E1
:10070000000E66EC2BF07AEF03F0086A28EC2BF071
:10071000400E34EC2BF0B90E4DEC2BF01DB805EF6C
:1007200005F01CB69FEF03F01CB8CDEF03F01CBA28
:10073000FBEF03F01CBC2BEF04F005EF05F0FF0E00
:1007400066EC2BF04DEC47F0FF0E66EC2BF04DEC19
:1007500048F0FF0E66EC2BF03DEC48F0FF0E66EC27
:100760002BF0FF0E66EC2BF0FF0E3DEC47F0FF0E7A
:1007700066EC2BF04DEC47F0FF0E66EC2BF0082AF0
:10078000110E085CD8B4CAEF03F0000E66EC2BF033
:10079000BFEF03F0086A11EF05F0FF0E66EC2BF0D7
:1007A0004DEC47F0FF0E66EC2BF04DEC48F0FF0EE1
:1007B00066EC2BF03DEC48F0FF0E66EC2BF0FF0EE4
:1007C00066EC2BF0FF0ECDEC47F0FF0E66EC2BF045
:1007D0004DEC47F0FF0E66EC2BF0082A110E085C7A
:1007E000D8B4F8EF03F0000E66EC2BF0EDEF03F059
:1007F000086A11EF05F0FF0E66EC2BF09DEC47F058
:10080000FF0E66EC2BF05DEC47F0FF0E66EC2BF074
:100810003DEC47F0FF0E66EC2BF0ADEC43F0FF0E25
:1008200066EC2BF05DEC43F0FF0E66EC2BF0DDEC9C
:1008300043F0FF0E66EC2BF07DEC43F0FF0E66EC10
:100840002BF0BDEC43F0FF0E66EC2BF0000E66ECD7
:100850002BF011EF05F0FF0E66EC2BF00DEC48F0DD
:10086000FF0E66EC2BF03DEC47F0FF0E66EC2BF034
:10087000DDEC47F0FF0E66EC2BF0000E66EC2BF083
:100880002B50526E529E010E525CD8B465EF04F0AC
:10089000490E525CD8B48DEF04F0030E525CD8B40C
:1008A000B5EF04F0430E525CD8B4DDEF04F0082A33
:1008B0001E0E085CD8B462EF04F0000E66EC2BF05C
:1008C00057EF04F0086A11EF05F0000E66EC2BF00C
:1008D000FF0E66EC2BF03DEC47F0FF0E66EC2BF0C4
:1008E0004DEC47F0FF0E66EC2BF0BDEC48F0000E2F
:1008F00066EC2BF0BDEC48F0000E66EC2BF0000E21
:1009000066EC2BF0000E66EC2BF0000E66EC2BF084
:10091000000E66EC2BF011EF05F0000E66EC2BF0EC
:10092000FF0E66EC2BF0DDEC47F0FF0E66EC2BF0D3
:100930004DEC47F0FF0E66EC2BF0BDEC48F0000EDE
:1009400066EC2BF0BDEC48F0000E66EC2BF0000ED0
:1009500066EC2BF0000E66EC2BF0000E66EC2BF034
:10096000000E66EC2BF011EF05F0000E66EC2BF09C
:10097000FF0E66EC2BF04DEC47F0FF0E66EC2BF013
:100980001DEC47F0FF0E66EC2BF04DEC48F0FF0E2F
:1009900066EC2BF0BDEC48F0000E66EC2BF0000E80
:1009A00066EC2BF0000E66EC2BF0000E66EC2BF0E4
:1009B000000E66EC2BF011EF05F0000E66EC2BF04C
:1009C000FF0E66EC2BF04DEC47F0FF0E66EC2BF0C3
:1009D0003DEC47F0FF0E66EC2BF03DEC47F0FF0ED0
:1009E00066EC2BF0BDEC48F0000E66EC2BF0000E30
:1009F00066EC2BF0000E66EC2BF0000E66EC2BF094
:100A0000000E66EC2BF011EF05F0082A320E085CA0
:100A1000D8B410EF05F0000E66EC2BF005EF05F0F2
:100A2000086A28EC2BF0730E34EC2BF0B90E4DEC69
:100A30002BF01DB84FEF05F01CA24FEF05F0FF0E95
:100A400066EC2BF03DEC48F0FF0E66EC2BF09DECD5
:100A500047F0FF0E66EC2BF02BEC2BF0400E34EC45
:100A60002BF0B90E4DEC2BF0CDEC47F0FF0E66EC01
:100A70002BF05DEC47F0FF0E66EC2BF0EDEC47F051
:100A8000FF0E66EC2BF03DEC47F0FF0E66EC2BF012
:100A90005DEC47F0FF0E66EC2BF06FEF05F0082AD7
:100AA0000E0E085CD8B45AEF05F0000E66EC2BF081
:100AB0004FEF05F0086A2BEC2BF0400E34EC2BF0D6
:100AC000B90E4DEC2BF0082A1F0E085CD8B46EEF5F
:100AD00005F0000E66EC2BF063EF05F0086A2BECD6
:100AE0002BF0600E34EC2BF0B90E4DEC2BF01DB852
:100AF0009FEF05F01CA09FEF05F0FF0E66EC2BF0BA
:100B00008DEC47F0FF0E66EC2BF09DEC47F0FF0EEE
:100B100066EC2BF0FF0E66EC2BF0FF0E66EC2BF074
:100B20006DEC47F0FF0E66EC2BF03DEC48F0FF0E4D
:100B300066EC2BF0000E66EC2BF0ABEF05F0082A0C
:100B40001C0E085CD8B4AAEF05F0000E66EC2BF082
:100B50009FEF05F0086A28EC2BF0400E34EC2BF0E8
:100B6000BB0E4DEC2BF04CB0BBEF05F01D504E6EA4
:100B70004F6AD0EF05F01D504E5CD8A43F9A000E8E
:100B80004F5CD8A4C6EF05F01D504E6E3FBAD0EFB3
:100B900005F0000E4E5CD8B4D0EF05F083EC3AF0CF
:100BA000000E4E5CD8A4D9EF05F001EC3BF023EF2A
:100BB00006F0400E4E5CD8A4E2EF05F021EC3BF0CD
:100BC00023EF06F0200E4E5CD8A4EBEF05F042ECCC
:100BD0003BF023EF06F0100E4E5CD8A4F4EF05F0C6
:100BE00063EC3BF023EF06F0080E4E5CD8A4FDEF5B
:100BF00005F09BEC3BF023EF06F0020E4E5CD8A410
:100C000006EF06F0E9EC3BF023EF06F0010E4E5C38
:100C1000D8A40FEF06F037EC3CF023EF06F0FF0E00
:100C200066EC2BF0B7EC3CF04E50B4EC39F0FF0E14
:100C300066EC2BF0FF0E66EC2BF016EC3AF0BDECF8
:100C400048F0BDEC48F028EC2BF0400E34EC2BF0D3
:100C5000BD0E4DEC2BF0000E66EC2BF0DDEC45F0FC
:100C6000000E66EC2BF09DEC46F0000E66EC2BF0CF
:100C7000280E66EC2BF0280E66EC2BF0280E66ECA6
:100C80002BF0280E66EC2BF0280E66EC2BF0000EF5
:100C900066EC2BF028EC2BF0530E34EC2BF0BD0E51
:100CA0004DEC2BF05E0E295CD8A476EF06F0000E1A
:100CB00066EC2BF0BDEC48F0000E66EC2BF0BDECC2
:100CC00048F0000E66EC2BF0000E66EC2BF0000EE8
:100CD00066EC2BF0DDEC42F0000E66EC2BF0CDEC78
:100CE00042F0000E66EC2BF09BEF08F05D0E295CE5
:100CF000D8A49AEF06F0000E66EC2BF0BDEC48F09D
:100D0000000E66EC2BF0BDEC48F0000E66EC2BF00C
:100D1000000E66EC2BF0000E66EC2BF0DDEC42F0E2
:100D2000000E66EC2BF0CDEC42F0000E66EC2BF0E2
:100D30009BEF08F0440E295CD8A4BEEF06F0000E2D
:100D400066EC2BF0BDEC48F0000E66EC2BF0EDEC01
:100D500042F0000E66EC2BF0EDEC42F0000E66EC7B
:100D60002BF0400E66EC2BF0000E66EC2BF0BDEC89
:100D700042F0000E66EC2BF09BEF08F0450E295C6C
:100D8000D8A4E2EF06F0000E66EC2BF0BDEC48F0C4
:100D9000000E66EC2BF0EDEC42F0000E66EC2BF052
:100DA000EDEC42F0000E66EC2BF0400E66EC2BF002
:100DB000000E66EC2BF0BDEC42F0000E66EC2BF062
:100DC0009BEF08F03E0E295CD8A406EF07F0000E5A
:100DD00066EC2BF0BDEC48F0000E66EC2BF0BDECA1
:100DE00048F0000E66EC2BF0000E66EC2BF0000EC7
:100DF00066EC2BF0EDEC42F0000E66EC2BF02DECE7
:100E000043F0000E66EC2BF09BEF08F03F0E295CE0
:100E1000D8A42AEF07F0000E66EC2BF0BDEC48F0EA
:100E2000000E66EC2BF0BDEC48F0000E66EC2BF0EB
:100E3000000E66EC2BF0000E66EC2BF0EDEC42F0B1
:100E4000000E66EC2BF02DEC43F0000E66EC2BF060
:100E50009BEF08F0220E295CD8A44EEF07F0000E9D
:100E600066EC2BF0BDEC48F0FF0E66EC2BF0CDEC01
:100E700043F0FF0E66EC2BF0CDEC43F0FF0E66EC7A
:100E80002BF0BF0E66EC2BF0FF0E66EC2BF06DEC3A
:100E900043F0FF0E66EC2BF09BEF08F0230E295C6D
:100EA000D8A472EF07F0000E66EC2BF0BDEC48F012
:100EB000FF0E66EC2BF0CDEC43F0FF0E66EC2BF052
:100EC000CDEC43F0FF0E66EC2BF0BF0E66EC2BF082
:100ED000FF0E66EC2BF06DEC43F0FF0E66EC2BF092
:100EE0009BEF08F01F0E295CD8A496EF07F0000EC8
:100EF00066EC2BF0BDEC48F0000E66EC2BF0BDEC80
:100F000048F0000E66EC2BF0000E66EC2BF0FF0EA6
:100F100066EC2BF0DDEC43F0FF0E66EC2BF0ADEC55
:100F200043F0FF0E66EC2BF09BEF08F0200E295CDF
:100F3000D8A4BAEF07F0000E66EC2BF0BDEC48F039
:100F4000000E66EC2BF0BDEC48F0000E66EC2BF0CA
:100F5000000E66EC2BF0FF0E66EC2BF0DDEC43F0A0
:100F6000FF0E66EC2BF0ADEC43F0FF0E66EC2BF0C1
:100F70009BEF08F0110E295CD8A4DEEF07F0FF0EFE
:100F800066EC2BF05DEC43F0FF0E66EC2BF0BDEC55
:100F900043F0FF0E66EC2BF0ADEC43F0FF0E66EC79
:100FA0002BF0BF0E66EC2BF0FF0E66EC2BF08DECF9
:100FB00043F0FF0E66EC2BF09BEF08F0120E295C5D
:100FC000D8A402EF08F0FF0E66EC2BF05DEC43F0C6
:100FD000FF0E66EC2BF0BDEC43F0FF0E66EC2BF041
:100FE000ADEC43F0FF0E66EC2BF0BF0E66EC2BF081
:100FF000FF0E66EC2BF08DEC43F0FF0E66EC2BF051
:101000009BEF08F0100E295CD8A426EF08F0000E24
:1010100066EC2BF0BDEC48F0000E66EC2BF0000EF9
:1010200066EC2BF0FF0E66EC2BF05DEC43F0FF0E50
:1010300066EC2BF0DDEC43F0FF0E66EC2BF06DEC74
:1010400043F0FF0E66EC2BF09BEF08F00F0E295CCF
:10105000D8A44AEF08F0000E66EC2BF0BDEC48F087
:10106000000E66EC2BF0000E66EC2BF0FF0E66EC2B
:101070002BF05DEC43F0FF0E66EC2BF0DDEC43F063
:10108000FF0E66EC2BF06DEC43F0FF0E66EC2BF0E0
:101090009BEF08F0000E66EC2BF0100E66EC2BF0C8
:1010A000100E66EC2BF0100E66EC2BF0100E66ECBA
:1010B0002BF0100E66EC2BF0000E66EC2BF0100EF1
:1010C00066EC2BF0100E66EC2BF0100E66EC2BF09D
:1010D000100E66EC2BF0100E66EC2BF0000E66EC9A
:1010E0002BF0100E66EC2BF0100E66EC2BF0100EB1
:1010F00066EC2BF0100E66EC2BF0100E66EC2BF06D
:10110000000E66EC2BF0400E66EC2BF0000E66EC49
:101110002BF0100E66EC2BF0100E66EC2BF0100E80
:1011200066EC2BF0100E66EC2BF0100E66EC2BF03C
:10113000000E66EC2BF0000E66EC2BF01DEC46F07A
:10114000000E66EC2BF0FDEC45F0000E66EC2BF08B
:101150000DEC47F0000E66EC2BF028EC2BF0400E67
:1011600034EC2BF0BC0E4DEC2BF0000E66EC2BF0AB
:101170000DEC46F0000E66EC2BF04DEC46F0000E48
:1011800066EC2BF0280E66EC2BF0280E66EC2BF0AC
:10119000280E66EC2BF0280E66EC2BF0280E66EC81
:1011A0002BF0000E66EC2BF028EC2BF0530E34ECF9
:1011B0002BF0BC0E4DEC2BF01550380B406E000E92
:1011C000405CD8A40CEF09F0000E66EC2BF08DEC1F
:1011D00046F0000E66EC2BF0EDEC46F0000E66ECEF
:1011E0002BF06DEC46F0000E66EC2BF0ADEC42F00F
:1011F000000E66EC2BF0BDEC48F0000E66EC2BF018
:10120000BDEC48F0000E66EC2BF0BDEC48F0000E93
:1012100066EC2BF057EF0AF0080E405CD8A439EFCB
:1012200009F0000E66EC2BF08DEC46F0000E66EC3B
:101230002BF0EDEC46F0000E66EC2BF06DEC46F07A
:10124000000E66EC2BF0BDEC42F0000E66EC2BF0CD
:10125000BDEC48F0000E66EC2BF0BDEC48F0000E43
:1012600066EC2BF0BDEC48F0000E66EC2BF057EF6F
:101270000AF0100E405CD8A466EF09F0000E66EC90
:101280002BF08DEC46F0000E66EC2BF0EDEC46F00A
:10129000000E66EC2BF06DEC46F0000E66EC2BF0C9
:1012A000CDEC42F0000E66EC2BF0BDEC48F0000EE9
:1012B00066EC2BF0BDEC48F0000E66EC2BF0BDECBC
:1012C00048F0000E66EC2BF057EF0AF0180E405C69
:1012D000D8A4AAEF09F0000E66EC2BF0BDEC46F0A6
:1012E000000E66EC2BF09DEC46F0000E66EC2BF049
:1012F0009DEC45F0000E66EC2BF0BDEC48F083A2AF
:1013000096EF09F0FF0E66EC2BF01DEC47F0FF0E98
:1013100066EC2BF03DEC47F0FF0E66EC2BF04DEC4D
:1013200048F0FF0E66EC2BF057EF0AF0000E66EC6B
:101330002BF09DEC46F0000E66EC2BF06DEC46F0C9
:10134000000E66EC2BF0BDEC45F0000E66EC2BF0C9
:1013500057EF0AF0200E405CD8A4D7EF09F0000E3A
:1013600066EC2BF08DEC46F0000E66EC2BF0EDEC0D
:1013700046F0000E66EC2BF06DEC46F0000E66ECCD
:101380002BF0EDEC42F0000E66EC2BF0BDEC48F0DB
:10139000000E66EC2BF0BDEC48F0000E66EC2BF076
:1013A000BDEC48F0000E66EC2BF057EF0AF0280E6B
:1013B000405CD8A404EF0AF0000E66EC2BF08DEC34
:1013C00046F0000E66EC2BF0EDEC46F0000E66ECFD
:1013D0002BF06DEC46F0000E66EC2BF0FDEC42F0CD
:1013E000000E66EC2BF0BDEC48F0000E66EC2BF026
:1013F000BDEC48F0000E66EC2BF0BDEC48F0000EA2
:1014000066EC2BF057EF0AF0300E405CD8A431EFB9
:101410000AF0000E66EC2BF08DEC46F0000E66EC48
:101420002BF0EDEC46F0000E66EC2BF06DEC46F088
:10143000000E66EC2BF00DEC43F0000E66EC2BF08A
:10144000BDEC48F0000E66EC2BF0BDEC48F0000E51
:1014500066EC2BF0BDEC48F0000E66EC2BF057EF7D
:101460000AF0000E66EC2BF08DEC46F0000E66ECF8
:101470002BF0EDEC46F0000E66EC2BF06DEC46F038
:10148000000E66EC2BF01DEC43F0000E66EC2BF02A
:10149000BDEC48F0000E66EC2BF0BDEC48F0000E01
:1014A00066EC2BF0BDEC48F0000E66EC2BF01DA8AE
:1014B00050921DB872EF0AF0020E1F5CD8B47EEF96
:1014C0000AF0030E1F5CD8B47EEF0AF0010E1F5C19
:1014D000D8B47EEF0AF0210E1F5CD8B47EEF0AF07C
:1014E00078EF0AF050B278EF0AF06DEC2CF05082F1
:1014F000206A216A226A236A266A276A2050D2EC6F
:1015000039F028EC2BF0400E34EC2BF0BE0E4DECF5
:101510002BF0080E66EC2BF0F80E66EC2BF0080EA4
:1015200066EC2BF0E00E66EC2BF0200E66EC2BF058
:10153000000E66EC2BF0000E66EC2BF0059CEEEC3A
:1015400039F02150D2EC39F028EC2BF05A0E34EC63
:101550002BF0BE0E4DEC2BF0F80E66EC2BF0000ECF
:1015600066EC2BF0E00E66EC2BF0200E66EC2BF018
:10157000E00E66EC2BF0000E66EC2BF0000E66EC35
:101580002BF0059CEEEC39F02250D2EC39F028EC2F
:101590002BF0400E34EC2BF0BF0E4DEC2BF0059CE5
:1015A000EEEC39F0DDEC48F02350D2EC39F028ECC9
:1015B0002BF04E0E34EC2BF0BF0E4DEC2BF0059CB7
:1015C000EEEC39F02650D2EC39F028EC2BF05C0E22
:1015D00034EC2BF0BF0E4DEC2BF0059CEEEC39F00B
:1015E000DDEC48F02750D2EC39F028EC2BF06A0EF5
:1015F00034EC2BF0BF0E4DEC2BF0059CEEEC39F0EB
:101600002BEC2BF0460E34EC2BF0BC0E4DEC2BF0FB
:10161000700E66EC2BF0100E66EC2BF0100E66ECE4
:101620002BF0100E66EC2BF0000E66EC2BF0EDECC0
:1016300045F0000E66EC2BF06DEC46F0000E66EC0B
:101640002BF05DEC46F0000E66EC2BF0082A220E23
:10165000085CD8B431EF0BF0100E66EC2BF026EFDF
:101660000BF0086A700E66EC2BF02BEC2BF0460E9C
:1016700034EC2BF0BD0E4DEC2BF0000E66EC2BF095
:10168000ADEC42F0000E66EC2BF0280E66EC2BF071
:10169000280E66EC2BF0280E66EC2BF0280E66EC7C
:1016A0002BF0280E66EC2BF0000E66EC2BF013509E
:1016B0000F0B406E02EC2FF02BEC2BF0460E34ECAF
:1016C0002BF0BE0E4DEC2BF0000E66EC2BF0BDECBB
:1016D00042F0000E66EC2BF0280E66EC2BF0280E84
:1016E00066EC2BF0280E66EC2BF0280E66EC2BF047
:1016F000280E66EC2BF0000E66EC2BF01450F00B6D
:10170000406E404240424042404202EC2FF02BECFF
:101710002BF0460E34EC2BF0BF0E4DEC2BF0000EF0
:1017200066EC2BF0CDEC42F0000E66EC2BF0280EB0
:1017300066EC2BF0280E66EC2BF0280E66EC2BF0F6
:10174000280E66EC2BF0280E66EC2BF0000E66ECF3
:101750002BF014500F0B406E02EC2FF023EF01F032
:101760004F6A28EC2BF0410E34EC2BF0B80E4DEC08
:101770002BF0700E66EC2BF0100E66EC2BF0100EBA
:1017800066EC2BF0100E66EC2BF0000E66EC2BF0E6
:10179000ADEC45F0000E66EC2BF09DEC46F0000E33
:1017A00066EC2BF02DEC43F0000E66EC2BF0EDEC2C
:1017B00042F0000E66EC2BF0BDEC42F0000E66EC41
:1017C0002BF00DEC43F0000E66EC2BF0BDEC48F076
:1017D0008DEC46F0000E66EC2BF0CDEC45F0000EE3
:1017E00066EC2BF0EDEC45F02BEC2BF0400E34ECDE
:1017F0002BF0B80E4DEC2BF0000E66EC2BF00DEC40
:1018000046F0000E66EC2BF09DEC46F0000E66EC08
:101810002BF0ADEC46F0000E66EC2BF0CDEC45F075
:10182000000E66EC2BF08DEC46F0000E66EC2BF013
:10183000082A200E085CD8B423EF0CF0100E66ECDA
:101840002BF018EF0CF0086A700E66EC2BF028EC09
:101850002BF0410E34EC2BF0B90E4DEC2BF0FF0EBB
:1018600066EC2BF01DEC47F0FF0E66EC2BF04DEC18
:1018700047F0FF0E66EC2BF04DEC47F0FF0E66ECE8
:101880002BF02DEC48F0FF0E66EC2BF05DEC47F0F2
:10189000FF0E66EC2BF03DEC48F0FF0E66EC2BF0F3
:1018A0003DEC48F0FF0E66EC2BF02BEC2BF0410EDC
:1018B00034EC2BF0B90E4DEC2BF0FF0E66EC2BF058
:1018C0004DEC47F0FF0E66EC2BF01DEC47F0FF0EE1
:1018D00066EC2BF04DEC48F0FF0E66EC2BF01DECA7
:1018E00047F0FF0E66EC2BF080B091EF0CF0070E86
:1018F000555CD8B47FEF0CF0552A93EF0CF0556A85
:101900003EB093EF0CF0060E425CD8B48BEF0CF0B7
:10191000422A8CEF0CF0426A50EC2CF03E8093EFA0
:101920000CF03E90556A84B6B1EF0CF0070E545C93
:10193000D8B49EEF0CF0542AB3EF0CF0546A3EBCBE
:10194000B3EF0CF0000E425CD8B4AAEF0CF04206E4
:10195000ACEF0CF0060E426E50EC2CF03E8CB3EF68
:101960000CF03E9C546A28EC2BF0410E34EC2BF02A
:10197000BA0E4DEC2BF0000E425CD8B4E0EF0CF048
:10198000010E425CD8B4A6EF0DF0020E425CD8B452
:101990006CEF0EF0030E425CD8B432EF0FF0040E81
:1019A000425CD8B4F8EF0FF0050E425CD8B4BEEF3D
:1019B00010F0060E425CD8B484EF11F0E2EF11F0A3
:1019C000ADEC42F0000E66EC2BF0ADEC42F0000EF8
:1019D00066EC2BF0FDEC45F0000E66EC2BF02BECEA
:1019E0002BF0410E34EC2BF0BA0E4DEC2BF01150D5
:1019F0002CEC3AF028EC2BF0410E34EC2BF0BB0E23
:101A00004DEC2BF0ADEC42F0000E66EC2BF0BDEC93
:101A100042F0000E66EC2BF0FDEC45F0000E66EC9B
:101A20002BF02BEC2BF0410E34EC2BF0BB0E4DECDD
:101A30002BF012502CEC3AF028EC2BF0410E34EC49
:101A40002BF0BC0E4DEC2BF0ADEC42F0000E66EC32
:101A50002BF0CDEC42F0000E66EC2BF0FDEC45F0E7
:101A6000000E66EC2BF02BEC2BF0410E34EC2BF03F
:101A7000BC0E4DEC2BF013502CEC3AF028EC2BF074
:101A8000410E34EC2BF0BD0E4DEC2BF0ADEC42F0E2
:101A9000000E66EC2BF0DDEC42F0000E66EC2BF055
:101AA000FDEC45F0000E66EC2BF02BEC2BF0410E1C
:101AB00034EC2BF0BD0E4DEC2BF014502CEC3AF026
:101AC00028EC2BF0410E34EC2BF0BE0E4DEC2BF03D
:101AD000ADEC42F0000E66EC2BF0EDEC42F0000EA7
:101AE00066EC2BF0FDEC45F0000E66EC2BF02BECD9
:101AF0002BF0410E34EC2BF0BE0E4DEC2BF01550BC
:101B00002CEC3AF028EC2BF0410E34EC2BF0BF0E0D
:101B10004DEC2BF0ADEC42F0000E66EC2BF0FDEC42
:101B200042F0000E66EC2BF0FDEC45F0000E66EC8A
:101B30002BF02BEC2BF0410E34EC2BF0BF0E4DECC8
:101B40002BF016502CEC3AF0E2EF11F0ADEC42F035
:101B5000000E66EC2BF00DEC43F0000E66EC2BF063
:101B6000FDEC45F0000E66EC2BF02BEC2BF0410E5B
:101B700034EC2BF0BA0E4DEC2BF017502CEC3AF065
:101B800028EC2BF0410E34EC2BF0BB0E4DEC2BF07F
:101B9000ADEC42F0000E66EC2BF01DEC43F0000EB5
:101BA00066EC2BF0FDEC45F0000E66EC2BF02BEC18
:101BB0002BF0410E34EC2BF0BB0E4DEC2BF01850FB
:101BC0002CEC3AF028EC2BF0410E34EC2BF0BC0E50
:101BD0004DEC2BF0ADEC42F0000E66EC2BF02DEC52
:101BE00043F0000E66EC2BF0FDEC45F0000E66ECC9
:101BF0002BF02BEC2BF0410E34EC2BF0BC0E4DEC0B
:101C00002BF019502CEC3AF028EC2BF0410E34EC70
:101C10002BF0BD0E4DEC2BF0ADEC42F0000E66EC5F
:101C20002BF03DEC43F0000E66EC2BF0FDEC45F0A4
:101C3000000E66EC2BF02BEC2BF0410E34EC2BF06D
:101C4000BD0E4DEC2BF01A502CEC3AF028EC2BF09A
:101C5000410E34EC2BF0BE0E4DEC2BF0ADEC42F00F
:101C6000000E66EC2BF08DEC45F0000E66EC2BF0D0
:101C7000FDEC45F0000E66EC2BF02BEC2BF0410E4A
:101C800034EC2BF0BE0E4DEC2BF01B502CEC3AF04C
:101C900028EC2BF0410E34EC2BF0BF0E4DEC2BF06A
:101CA000ADEC42F0000E66EC2BF09DEC45F0000E22
:101CB00066EC2BF0FDEC45F0000E66EC2BF02BEC07
:101CC0002BF0410E34EC2BF0BF0E4DEC2BF01C50E2
:101CD0002CEC3AF0E2EF11F0ADEC42F0000E66ECC5
:101CE0002BF0ADEC45F0000E66EC2BF0FDEC45F072
:101CF000000E66EC2BF02BEC2BF0410E34EC2BF0AD
:101D0000BA0E4DEC2BF01D502CEC3AF028EC2BF0D9
:101D1000410E34EC2BF0BB0E4DEC2BF0ADEC42F051
:101D2000000E66EC2BF0BDEC45F0000E66EC2BF0DF
:101D3000FDEC45F0000E66EC2BF02BEC2BF0410E89
:101D400034EC2BF0BB0E4DEC2BF01E502CEC3AF08B
:101D500028EC2BF0410E34EC2BF0BC0E4DEC2BF0AC
:101D6000ADEC42F0000E66EC2BF0CDEC45F0000E31
:101D700066EC2BF0FDEC45F0000E66EC2BF02BEC46
:101D80002BF0410E34EC2BF0BC0E4DEC2BF01F5021
:101D90002CEC3AF028EC2BF0410E34EC2BF0BD0E7D
:101DA0004DEC2BF0ADEC42F0000E66EC2BF0DDECD0
:101DB00045F0000E66EC2BF0FDEC45F0000E66ECF5
:101DC0002BF02BEC2BF0410E34EC2BF0BD0E4DEC38
:101DD0002BF020502CEC3AF028EC2BF0410E34EC98
:101DE0002BF0BE0E4DEC2BF0BDEC42F0000E66EC7D
:101DF0002BF0ADEC42F0000E66EC2BF0FDEC45F064
:101E0000000E66EC2BF02BEC2BF0410E34EC2BF09B
:101E1000BE0E4DEC2BF021502CEC3AF028EC2BF0C0
:101E2000410E34EC2BF0BF0E4DEC2BF0BDEC42F02C
:101E3000000E66EC2BF0BDEC42F0000E66EC2BF0D1
:101E4000FDEC45F0000E66EC2BF02BEC2BF0410E78
:101E500034EC2BF0BF0E4DEC2BF022502CEC3AF072
:101E6000E2EF11F0BDEC42F0000E66EC2BF0CDEC91
:101E700042F0000E66EC2BF0FDEC45F0000E66EC37
:101E80002BF02BEC2BF0410E34EC2BF0BA0E4DEC7A
:101E90002BF023502CEC3AF028EC2BF0410E34ECD4
:101EA0002BF0BB0E4DEC2BF0BDEC42F0000E66ECBF
:101EB0002BF0DDEC42F0000E66EC2BF0FDEC45F073
:101EC000000E66EC2BF02BEC2BF0410E34EC2BF0DB
:101ED000BB0E4DEC2BF024502CEC3AF028EC2BF000
:101EE000410E34EC2BF0BC0E4DEC2BF0BDEC42F06F
:101EF000000E66EC2BF0EDEC42F0000E66EC2BF0E1
:101F0000FDEC45F0000E66EC2BF02BEC2BF0410EB7
:101F100034EC2BF0BC0E4DEC2BF025502CEC3AF0B1
:101F200028EC2BF0410E34EC2BF0BD0E4DEC2BF0D9
:101F3000BDEC42F0000E66EC2BF0FDEC42F0000E22
:101F400066EC2BF0FDEC45F0000E66EC2BF02BEC74
:101F50002BF0410E34EC2BF0BD0E4DEC2BF0265047
:101F60002CEC3AF028EC2BF0410E34EC2BF0BE0EAA
:101F70004DEC2BF0BDEC42F0000E66EC2BF00DECBE
:101F800043F0000E66EC2BF0FDEC45F0000E66EC25
:101F90002BF02BEC2BF0410E34EC2BF0BE0E4DEC65
:101FA0002BF027502CEC3AF028EC2BF0410E34ECBF
:101FB0002BF0BF0E4DEC2BF0BDEC42F0000E66ECAA
:101FC0002BF01DEC43F0000E66EC2BF0FDEC45F021
:101FD000000E66EC2BF02BEC2BF0410E34EC2BF0CA
:101FE000BF0E4DEC2BF028502CEC3AF0E2EF11F044
:101FF000BDEC42F0000E66EC2BF02DEC43F0000E31
:1020000066EC2BF0FDEC45F0000E66EC2BF02BECB3
:102010002BF0410E34EC2BF0BA0E4DEC2BF0295086
:102020002CEC3AF028EC2BF0410E34EC2BF0BB0EEC
:102030004DEC2BF0BDEC42F0000E66EC2BF03DECCD
:1020400043F0000E66EC2BF0FDEC45F0000E66EC64
:102050002BF02BEC2BF0410E34EC2BF0BB0E4DECA7
:102060002BF02A502CEC3AF028EC2BF0410E34ECFB
:102070002BF0BC0E4DEC2BF0BDEC42F0000E66ECEC
:102080002BF08DEC45F0000E66EC2BF0FDEC45F0EE
:10209000000E66EC2BF02BEC2BF0410E34EC2BF009
:1020A000BC0E4DEC2BF02B502CEC3AF028EC2BF026
:1020B000410E34EC2BF0BD0E4DEC2BF0BDEC42F09C
:1020C000000E66EC2BF09DEC45F0000E66EC2BF05C
:1020D000FDEC45F0000E66EC2BF02BEC2BF0410EE6
:1020E00034EC2BF0BD0E4DEC2BF02C502CEC3AF0D8
:1020F00028EC2BF0410E34EC2BF0BE0E4DEC2BF007
:10210000BDEC42F0000E66EC2BF0ADEC45F0000E9D
:1021100066EC2BF0FDEC45F0000E66EC2BF02BECA2
:102120002BF0410E34EC2BF0BE0E4DEC2BF02D506D
:102130002CEC3AF028EC2BF0410E34EC2BF0BF0ED7
:102140004DEC2BF0BDEC42F0000E66EC2BF0BDEC3C
:1021500045F0000E66EC2BF0FDEC45F0000E66EC51
:102160002BF02BEC2BF0410E34EC2BF0BF0E4DEC92
:102170002BF02E502CEC3AF0E2EF11F0BDEC42F0D7
:10218000000E66EC2BF0CDEC45F0000E66EC2BF06B
:10219000FDEC45F0000E66EC2BF02BEC2BF0410E25
:1021A00034EC2BF0BA0E4DEC2BF02F502CEC3AF017
:1021B00028EC2BF0410E34EC2BF0BB0E4DEC2BF049
:1021C000BDEC42F0000E66EC2BF0DDEC45F0000EAD
:1021D00066EC2BF0FDEC45F0000E66EC2BF02BECE2
:1021E0002BF0410E34EC2BF0BB0E4DEC2BF03050AD
:1021F0002CEC3AF028EC2BF0410E34EC2BF0BC0E1A
:102200004DEC2BF0CDEC42F0000E66EC2BF0ADEC7B
:1022100042F0000E66EC2BF0FDEC45F0000E66EC93
:102220002BF02BEC2BF0410E34EC2BF0BC0E4DECD4
:102230002BF031502CEC3AF028EC2BF0410E34EC22
:102240002BF0BD0E4DEC2BF0CDEC42F0000E66EC09
:102250002BF0BDEC42F0000E66EC2BF0FDEC45F0EF
:10226000000E66EC2BF02BEC2BF0410E34EC2BF037
:10227000BD0E4DEC2BF032502CEC3AF028EC2BF04C
:10228000410E34EC2BF0BE0E4DEC2BF0CDEC42F0B9
:10229000000E66EC2BF0CDEC42F0000E66EC2BF05D
:1022A000FDEC45F0000E66EC2BF02BEC2BF0410E14
:1022B00034EC2BF0BE0E4DEC2BF033502CEC3AF0FE
:1022C00028EC2BF0410E34EC2BF0BF0E4DEC2BF034
:1022D000CDEC42F0000E66EC2BF0DDEC42F0000E8F
:1022E00066EC2BF0FDEC45F0000E66EC2BF02BECD1
:1022F0002BF0410E34EC2BF0BF0E4DEC2BF0345094
:102300002CEC3AF0E2EF11F0CDEC42F0000E66EC6E
:102310002BF0EDEC42F0000E66EC2BF0FDEC45F0FE
:10232000000E66EC2BF02BEC2BF0410E34EC2BF076
:10233000BA0E4DEC2BF035502CEC3AF028EC2BF08B
:10234000410E34EC2BF0BB0E4DEC2BF0CDEC42F0FB
:10235000000E66EC2BF0FDEC42F0000E66EC2BF06C
:10236000FDEC45F0000E66EC2BF02BEC2BF0410E53
:1023700034EC2BF0BB0E4DEC2BF036502CEC3AF03D
:1023800028EC2BF0410E34EC2BF0BC0E4DEC2BF076
:10239000CDEC42F0000E66EC2BF00DEC43F0000E9D
:1023A00066EC2BF0FDEC45F0000E66EC2BF02BEC10
:1023B0002BF0410E34EC2BF0BC0E4DEC2BF03750D3
:1023C0002CEC3AF0E9EC2EF023EF01F028EC2BF0A6
:1023D000410E34EC2BF0B80E4DEC2BF0700E66EC89
:1023E0002BF0100E66EC2BF0100E66EC2BF0100E9E
:1023F00066EC2BF0000E66EC2BF0ADEC45F0000E19
:1024000066EC2BF09DEC46F0000E66EC2BF02DEC0C
:1024100043F0000E66EC2BF0EDEC42F0000E66ECA3
:102420002BF0BDEC42F0000E66EC2BF00DEC43F00F
:10243000000E66EC2BF0BDEC48F09DEC46F0000E73
:1024400066EC2BF0CDEC45F0000E66EC2BF0ADEC1D
:1024500046F02BEC2BF0400E34EC2BF0B80E4DEC8C
:102460002BF0000E66EC2BF0ADEC46F0000E66ECA7
:102470002BF00DEC46F0000E66EC2BF04DEC46F028
:10248000000E66EC2BF0EDEC45F0000E66EC2BF048
:10249000082A260E085CD8B453EF12F0100E66EC32
:1024A0002BF048EF12F0086A700E66EC2BF0000E6D
:1024B000435CD8B463EF12F0010E435CD8B4A3EFD1
:1024C00015F023EF01F028EC2BF0460E34EC2BF046
:1024D000B90E4DEC2BF09DEC46F0000E66EC2BF0A7
:1024E000CDEC45F0000E66EC2BF02DEC46F0000E26
:1024F00066EC2BF0CDEC45F0000E66EC2BF0ADEC6D
:1025000045F0000E66EC2BF0ADEC46F0000E66ECEC
:102510002BF0BDEC48F08DEC45F0000E66EC2BF096
:10252000BDEC45F0000E66EC2BF0BDEC45F02BEC5D
:102530002BF0400E34EC2BF0B90E4DEC2BF0000ECE
:1025400066EC2BF08DEC46F0000E66EC2BF0CDEC3B
:1025500045F0000E66EC2BF09DEC46F0000E66ECAC
:102560002BF09DEC46F0000E66EC2BF080B0D1EF26
:1025700012F0070E555CD8B4C1EF12F0552AD3EF14
:1025800012F0556A3EB0D3EF12F00A0E465CD8B492
:10259000CDEF12F0462ACEEF12F0466A3E80D3EF1E
:1025A00012F03E90556A84B6EFEF12F0070E545CBD
:1025B000D8B4DEEF12F0542AF1EF12F0546A3EBCA8
:1025C000F1EF12F0000E465CD8B4EAEF12F04606C6
:1025D000ECEF12F00A0E466E3E8CF1EF12F03E9CCC
:1025E000546A3F9428EC2BF04A0E34EC2BF0BB0ECF
:1025F0004DEC2BF0000E465CD8B413EF13F0000E38
:1026000066EC2BF0ADEC42F0000E66EC2BF0ADEC7E
:1026100042F0000E66EC2BF0FDEC45F0000E66EC8F
:102620002BF025EF13F0FF0E66EC2BF04DEC43F092
:10263000FF0E66EC2BF04DEC43F0FF0E66EC2BF03A
:102640008DEC47F0FF0E66EC2BF028EC2BF0670EBC
:1026500034EC2BF0BB0E4DEC2BF0010E465CD8B4E5
:1026600046EF13F0000E66EC2BF0ADEC42F0000EDE
:1026700066EC2BF0BDEC42F0000E66EC2BF0FDECAE
:1026800045F0000E66EC2BF058EF13F0FF0E66ECF1
:102690002BF04DEC43F0FF0E66EC2BF05DEC43F0BD
:1026A000FF0E66EC2BF08DEC47F0FF0E66EC2BF086
:1026B0002BEC2BF0440E34EC2BF0BB0E4DEC2BF03E
:1026C000020E465CD8B479EF13F0000E66EC2BF0E6
:1026D000ADEC42F0000E66EC2BF0CDEC42F0000EBB
:1026E00066EC2BF0FDEC45F0000E66EC2BF08BEF6A
:1026F00013F0FF0E66EC2BF04DEC43F0FF0E66EC92
:102700002BF06DEC43F0FF0E66EC2BF08DEC47F0F8
:10271000FF0E66EC2BF02BEC2BF0610E34EC2BF063
:10272000BB0E4DEC2BF0030E465CD8B4ACEF13F0AF
:10273000000E66EC2BF0ADEC42F0000E66EC2BF0D8
:10274000DDEC42F0000E66EC2BF0FDEC45F0000EE7
:1027500066EC2BF0BEEF13F0FF0E66EC2BF04DECA9
:1027600043F0FF0E66EC2BF07DEC43F0FF0E66ECC1
:102770002BF08DEC47F0FF0E66EC2BF028EC2BF0E5
:102780004A0E34EC2BF0BC0E4DEC2BF0040E465CE4
:10279000D8B4DFEF13F0000E66EC2BF0ADEC42F096
:1027A000000E66EC2BF0EDEC42F0000E66EC2BF028
:1027B000FDEC45F0000E66EC2BF0F1EF13F0FF0E90
:1027C00066EC2BF04DEC43F0FF0E66EC2BF08DEC3D
:1027D00043F0FF0E66EC2BF08DEC47F0FF0E66EC3D
:1027E0002BF028EC2BF0670E34EC2BF0BC0E4DECEC
:1027F0002BF0050E465CD8B412EF14F0000E66EC18
:102800002BF0ADEC42F0000E66EC2BF0FDEC42F04C
:10281000000E66EC2BF0FDEC45F0000E66EC2BF0A4
:1028200024EF14F0FF0E66EC2BF04DEC43F0FF0E9E
:1028300066EC2BF09DEC43F0FF0E66EC2BF08DEC7C
:1028400047F0FF0E66EC2BF02BEC2BF0440E34EC33
:102850002BF0BC0E4DEC2BF0060E465CD8B445EFC9
:1028600014F0000E66EC2BF0ADEC42F0000E66ECBE
:102870002BF00DEC43F0000E66EC2BF0FDEC45F078
:10288000000E66EC2BF057EF14F0FF0E66EC2BF009
:102890004DEC43F0FF0E66EC2BF0ADEC43F0FF0E79
:1028A00066EC2BF08DEC47F0FF0E66EC2BF02BEC7A
:1028B0002BF0610E34EC2BF0B40E4DEC2BF0070E28
:1028C000465CD8B478EF14F0000E66EC2BF0ADEC5B
:1028D00042F0000E66EC2BF01DEC43F0000E66ECAF
:1028E0002BF0FDEC45F0000E66EC2BF08AEF14F0B7
:1028F000FF0E66EC2BF04DEC43F0FF0E66EC2BF078
:10290000BDEC43F0FF0E66EC2BF08DEC47F0FF0EB4
:1029100066EC2BF028EC2BF04A0E34EC2BF0BD0EBD
:102920004DEC2BF0080E465CD8B4ABEF14F0000E63
:1029300066EC2BF0ADEC42F0000E66EC2BF02DECCB
:1029400043F0000E66EC2BF0FDEC45F0000E66EC5B
:102950002BF0BDEF14F0FF0E66EC2BF04DEC43F0C6
:10296000FF0E66EC2BF0CDEC43F0FF0E66EC2BF087
:102970008DEC47F0FF0E66EC2BF028EC2BF0670E89
:1029800034EC2BF0BD0E4DEC2BF0090E465CD8B4A8
:10299000DEEF14F0000E66EC2BF0ADEC42F0000E12
:1029A00066EC2BF03DEC43F0000E66EC2BF0FDECFA
:1029B00045F0000E66EC2BF0F0EF14F0FF0E66EC25
:1029C0002BF04DEC43F0FF0E66EC2BF0DDEC43F00A
:1029D000FF0E66EC2BF08DEC47F0FF0E66EC2BF053
:1029E00028EC2BF04A0E34EC2BF0BF0E4DEC2BF004
:1029F0000A0E465CD8B443EF15F0000E66EC2BF0DF
:102A0000BDEC45F0000E66EC2BF0CDEC45F0000E71
:102A100066EC2BF0DDEC45F0000E66EC2BF08DEC57
:102A200045F0000E66EC2BF0BDEC46F0000E66ECB7
:102A30002BF02DEC46F0000E66EC2BF0ADEC46F0E2
:102A4000000E66EC2BF0BDEC48F02DEC46F0000ECD
:102A500066EC2BF02BEC2BF0400E34EC2BF0BF0E81
:102A60004DEC2BF05DEC46F0000E66EC2BF08DEC9F
:102A700045F0000E66EC2BF0BDEC45F0000E66EC68
:102A80002BF087EF15F0FF0E66EC2BF04DEC47F0C6
:102A9000FF0E66EC2BF05DEC47F0FF0E66EC2BF0C2
:102AA0006DEC47F0FF0E66EC2BF01DEC47F0FF0ECF
:102AB00066EC2BF05DEC48F0FF0E66EC2BF0CDECF5
:102AC00047F0FF0E66EC2BF04DEC48F0FF0E66EC85
:102AD0002BF0CDEC48F0CDEC47F0FF0E66EC2BF080
:102AE0002BEC2BF0400E34EC2BF0BF0E4DEC2BF00A
:102AF000FDEC47F0FF0E66EC2BF01DEC47F0FF0EEF
:102B000066EC2BF04DEC47F0FF0E66EC2BF0E9EC99
:102B10002EF080B89FEF15F0070E575CD8B494EFF5
:102B200015F0572AA1EF15F0576A3EB8A1EF15F03E
:102B3000010E436E50EC2CF03E88A1EF15F03E984C
:102B4000576A23EF01F028EC2BF0460E34EC2BF003
:102B5000B90E4DEC2BF0000E465CD8B4DFEF15F04B
:102B6000010E465CD8B4E0EF16F0020E465CD8B415
:102B700039EF18F0030E465CD8B44DEF19F0040E8F
:102B8000465CD8B431EF1AF0050E465CD8B440EF7D
:102B90001BF0060E465CD8B467EF1CF0070E465CCF
:102BA000D8B4CBEF1DF0080E465CD8B483EF1EF00E
:102BB000090E465CD8B43BEF1FF0F3EF1FF0FAECC0
:102BC0003CF03FB2E6EF15F0050E496E3FB449EF19
:102BD00016F080B017EF16F0070E555CD8B4F4EF7E
:102BE00015F0552A19EF16F0556A3EB019EF16F098
:102BF000010E495CD8A401EF16F0080E496E14EFDF
:102C000016F0040E495CD8A40AEF16F0010E496EC6
:102C100014EF16F0080E495CD8A413EF16F0050E59
:102C2000496E14EF16F049063E8019EF16F03E90FB
:102C3000556A84B647EF16F0070E545CD8B424EFFB
:102C400016F0542A49EF16F0546A3EBC49EF16F0CC
:102C5000080E495CD8A431EF16F0010E496E44EF1E
:102C600016F0010E495CD8A43AEF16F0040E496E36
:102C700044EF16F0050E495CD8A443EF16F0080E99
:102C8000496E44EF16F0492A3E8C49EF16F03E9CFF
:102C9000546A28EC2BF0460E34EC2BF0BC0E4DECB5
:102CA0002BF0010E495CD8B483EF16F0040E495C9A
:102CB000D8B4A6EF16F0080E495CD8B4C7EF16F0EA
:102CC000FF0E66EC2BF04DEC48F0FF0E66EC2BF09F
:102CD0002DEC48F0FF0E66EC2BF05DEC48F0FF0E9B
:102CE00066EC2BF0EDEC47F0FF0E66EC2BF03DECC4
:102CF00047F0FF0E66EC2BF0BDEC48F0000E66ECE2
:102D00002BF0C7EF16F0FF0E66EC2BF06DEC47F0E2
:102D1000FF0E66EC2BF03DEC48F0FF0E66EC2BF05E
:102D20007DEC48F0FF0E66EC2BF03DEC47F0FF0E1B
:102D300066EC2BF0CDEC47F0FF0E66EC2BF0BDEC13
:102D400047F0FF0E66EC2BF0C7EF16F0FF0E66ECB7
:102D50002BF00DEC48F0FF0E66EC2BF04DEC47F03D
:102D6000FF0E66EC2BF05DEC48F0FF0E66EC2BF0EE
:102D70002DEC48F0FF0E66EC2BF0BDEC48F0000E99
:102D800066EC2BF0BDEC48F0000E66EC2BF03FB685
:102D9000CEEF16F03F8611504A6E4B6E97EC32F034
:102DA0002BEC2BF0400E34EC2BF0BD0E4DEC2BF049
:102DB000405044EC3AF08DEC3AF03F82FEEF20F0C8
:102DC00053EC3DF03FB2E7EF16F0070E496E3FA41B
:102DD0001DEC32F028EC2BF0460E34EC2BF0BC0E40
:102DE0004DEC2BF0000E495CD8B442EF17F0010E09
:102DF000495CD8B46AEF17F0020E495CD8B492EF80
:102E000017F0030E495CD8B492EF17F0040E495C3A
:102E1000D8B4C6EF17F0050E495CD8B4C6EF17F06A
:102E2000060E495CD8B4FAEF17F0080E495CD8B426
:102E300020EF18F0FF0E66EC2BF03DEC47F0FF0E94
:102E400066EC2BF08DEC47F0FF0E66EC2BF03DECC2
:102E500048F0FF0E66EC2BF0BDEC48F0000E66EC7F
:102E60002BF0BDEC48F0000E66EC2BF0BDEC48F00A
:102E7000000E66EC2BF0BDEC48F0000E66EC2BF07B
:102E800020EF18F0FF0E66EC2BF03DEC48F0FF0E43
:102E900066EC2BF07DEC48F0FF0E66EC2BF03DEC81
:102EA00047F0FF0E66EC2BF0CDEC47F0FF0E66EC22
:102EB0002BF0BDEC47F0FF0E66EC2BF0BDEC48F0BC
:102EC000000E66EC2BF0BDEC48F0000E66EC2BF02B
:102ED00020EF18F0FF0E66EC2BF0DDEC47F0FF0E54
:102EE00066EC2BF05DEC48F0FF0E66EC2BF04DEC41
:102EF00048F0FF0E66EC2BF05DEC47F0FF0E66EC41
:102F00002BF03DEC48F0FF0E66EC2BF01DEC47F08B
:102F1000FF0E66EC2BF0FDEC47F0FF0E66EC2BF09D
:102F200020EF18F0FF0E66EC2BF09DEC47F0FF0E43
:102F300066EC2BF0EDEC47F0FF0E66EC2BF04DEC61
:102F400048F0FF0E66EC2BF0020E495CD8B4B0EFEF
:102F500017F04DEC43F0FF0E66EC2BF0B5EF17F0D9
:102F60005DEC43F0FF0E66EC2BF0BDEC48F0000E7C
:102F700066EC2BF0BDEC48F0000E66EC2BF0BDECDF
:102F800048F0000E66EC2BF020EF18F0FF0E66EC18
:102F90002BF08DEC47F0FF0E66EC2BF0FDEC47F0CC
:102FA000FF0E66EC2BF0CDEC47F0FF0E66EC2BF03D
:102FB0004DEC47F0FF0E66EC2BF0040E495CD8B4E4
:102FC000E9EF17F04DEC43F0FF0E66EC2BF0EEEF5F
:102FD00017F05DEC43F0FF0E66EC2BF0BDEC48F013
:102FE000000E66EC2BF0BDEC48F0000E66EC2BF00A
:102FF00020EF18F0FF0E66EC2BF02DEC48F0FF0EE2
:1030000066EC2BF0DDEC47F0FF0E66EC2BF03DECB0
:1030100047F0FF0E66EC2BF0BDEC47F0FF0E66ECC0
:103020002BF06DEC47F0FF0E66EC2BF0BDEC48F09A
:10303000000E66EC2BF0BDEC48F0000E66EC2BF0B9
:103040003FB627EF18F03F8612504A6E4B6E97EC52
:1030500032F02BEC2BF0400E34EC2BF0BD0E4DEC8F
:103060002BF0405044EC3AF08DEC3AF03F82FEEF0A
:1030700020F0ACEC3DF03FB240EF18F0070E496E87
:103080003FA41DEC32F028EC2BF0460E34EC2BF074
:10309000BC0E4DEC2BF0000E495CD8B4BAEF18F022
:1030A000010E495CD8B4ECEF18F0020E495CD8B4BC
:1030B000ECEF18F0030E495CD8B4ECEF18F0080EF2
:1030C000495CD8B434EF19F0FF0E66EC2BF07DECC0
:1030D00047F0FF0E66EC2BF00DEC48F0FF0E66ECAF
:1030E0002BF0FDEC47F0FF0E66EC2BF04DEC43F0BF
:1030F000FF0E66EC2BF03DEC48F0FF0E66EC2BF07B
:103100005DEC47F0FF0E66EC2BF0CDEC47F0FF0EC8
:1031100066EC2BF0040E495CD8B4A0EF18F0050E55
:10312000495CD8B4A7EF18F0060E495CD8B4AEEFEE
:1031300018F04DEC43F0FF0E66EC2BF0B3EF18F0F7
:103140007DEC43F0FF0E66EC2BF0B3EF18F06DEC66
:1031500043F0FF0E66EC2BF0B3EF18F05DEC43F09C
:10316000FF0E66EC2BF0BDEC48F0000E66EC2BF089
:1031700034EF19F0FF0E66EC2BF04DEC47F0FF0E2C
:1031800066EC2BF05DEC47F0FF0E66EC2BF04DEC9F
:1031900048F0FF0E66EC2BF03DEC47F0FF0E66ECBE
:1031A0002BF09DEC47F0FF0E66EC2BF0BDEC48F0E9
:1031B000000E66EC2BF0BDEC48F0000E66EC2BF038
:1031C000BDEC48F0000E66EC2BF0BDEC48F0000EB4
:1031D00066EC2BF034EF19F0FF0E66EC2BF05DEC93
:1031E00047F0FF0E66EC2BF0DDEC47F0FF0E66ECCF
:1031F0002BF00DEC48F0FF0E66EC2BF08DEC47F059
:10320000FF0E66EC2BF03DEC47F0FF0E66EC2BF06A
:10321000EDEC47F0FF0E66EC2BF04DEC48F0FF0EA6
:1032200066EC2BF0CDEC47F0FF0E66EC2BF0010EB8
:10323000495CD8B428EF19F0020E495CD8B42FEFDE
:1032400019F04DEC43F0FF0E66EC2BF034EF19F063
:103250006DEC43F0FF0E66EC2BF034EF19F05DECF3
:1032600043F0FF0E66EC2BF03FB63BEF19F03F86C4
:1032700013504A6E4B6E97EC32F02BEC2BF0400E55
:1032800034EC2BF0BD0E4DEC2BF0405044EC3AF0FA
:103290008DEC3AF03F82FEEF20F005EC3EF03FB2BD
:1032A00054EF19F0070E496E3FA41DEC32F028ECE4
:1032B0002BF0460E34EC2BF0BC0E4DEC2BF0000E38
:1032C000495CD8B4C9EF19F0010E495CD8B4C9EF14
:1032D00019F0020E495CD8B4C9EF19F0030E495C2D
:1032E000D8B4C9EF19F0080E495CD8B418EF1AF039
:1032F000FF0E66EC2BF07DEC47F0FF0E66EC2BF03A
:103300000DEC48F0FF0E66EC2BF0FDEC47F0FF0EE5
:1033100066EC2BF06DEC43F0FF0E66EC2BF03DEC11
:1033200048F0FF0E66EC2BF05DEC47F0FF0E66EC0C
:103330002BF0CDEC47F0FF0E66EC2BF0040E495C51
:10334000D8B4B4EF19F0050E495CD8B4BBEF19F04E
:10335000060E495CD8B4C2EF19F04DEC43F0FF0EF5
:1033600066EC2BF018EF1AF07DEC43F0FF0E66ECE4
:103370002BF018EF1AF06DEC43F0FF0E66EC2BF01B
:1033800018EF1AF05DEC43F0FF0E66EC2BF018EF2F
:103390001AF0FF0E66EC2BF07DEC47F0FF0E66ECAA
:1033A0002BF00DEC48F0FF0E66EC2BF0FDEC47F037
:1033B000FF0E66EC2BF05DEC43F0FF0E66EC2BF09D
:1033C0003DEC48F0FF0E66EC2BF05DEC47F0FF0E95
:1033D00066EC2BF0CDEC47F0FF0E66EC2BF0000E08
:1033E000495CD8B405EF1AF0010E495CD8B40CEF73
:1033F0001AF0020E495CD8B413EF1AF04DEC43F00A
:10340000FF0E66EC2BF018EF1AF07DEC43F0FF0E88
:1034100066EC2BF018EF1AF06DEC43F0FF0E66EC43
:103420002BF018EF1AF05DEC43F0FF0E66EC2BF07A
:103430003FB61FEF1AF03F8614504A6E4B6E97EC62
:1034400032F02BEC2BF0400E34EC2BF0BD0E4DEC9B
:103450002BF0405044EC3AF08DEC3AF03F82FEEF16
:1034600020F05EEC3EF03FB238EF1AF0070E496EE6
:103470003FA41DEC32F028EC2BF0460E34EC2BF080
:10348000BC0E4DEC2BF0000E495CD8B46DEF1AF079
:10349000010E495CD8B490EF1AF0020E495CD8B422
:1034A000B3EF1AF0030E495CD8B4B3EF1AF0040E70
:1034B000495CD8B4B3EF1AF0050E495CD8B4EEEF0E
:1034C0001AF0060E495CD8B4EEEF1AF0080E495C0B
:1034D000D8B427EF1BF0EEEF1AF0FF0E66EC2BF0DE
:1034E0002DEC48F0FF0E66EC2BF05DEC48F0FF0E83
:1034F00066EC2BF0EDEC47F0FF0E66EC2BF0BDEC2C
:1035000048F0000E66EC2BF0BDEC48F0000E66ECC7
:103510002BF0BDEC48F0000E66EC2BF027EF1BF013
:10352000FF0E66EC2BF02DEC48F0FF0E66EC2BF056
:103530008DEC48F0FF0E66EC2BF04DEC47F0FF0EE3
:1035400066EC2BF0BDEC48F0000E66EC2BF0BDEC09
:1035500048F0000E66EC2BF0BDEC48F0000E66EC77
:103560002BF027EF1BF0FF0E66EC2BF02DEC48F054
:10357000FF0E66EC2BF08DEC48F0FF0E66EC2BF0A6
:103580003DEC48F0FF0E66EC2BF05DEC47F0FF0ED3
:1035900066EC2BF0CDEC47F0FF0E66EC2BF0020E44
:1035A000495CD8B4E0EF1AF0030E495CD8B4E7EFF9
:1035B0001AF04DEC43F0FF0E66EC2BF027EF1BF0FA
:1035C0006DEC43F0FF0E66EC2BF027EF1BF05DEC8B
:1035D00043F0FF0E66EC2BF027EF1BF0FF0E66ECBE
:1035E0002BF04DEC48F0FF0E66EC2BF08DEC48F024
:1035F000FF0E66EC2BF03DEC48F0FF0E66EC2BF076
:103600005DEC47F0FF0E66EC2BF0CDEC47F0FF0EC3
:1036100066EC2BF0050E495CD8B41BEF1BF0060ED0
:10362000495CD8B422EF1BF04DEC43F0FF0E66EC82
:103630002BF027EF1BF06DEC43F0FF0E66EC2BF048
:1036400027EF1BF05DEC43F0FF0E66EC2BF03FB66E
:103650002EEF1BF03F8615504A6E4B6E97EC32F002
:103660002BEC2BF0400E34EC2BF0BD0E4DEC2BF080
:10367000405044EC3AF08DEC3AF03F82FEEF20F0FF
:10368000B7EC3EF03FB247EF1BF0070E496E3FA488
:103690001DEC32F028EC2BF0460E34EC2BF0BC0E77
:1036A0004DEC2BF0080E495CD8B44EEF1CF0FF0E29
:1036B00066EC2BF03DEC48F0FF0E66EC2BF0FDECD9
:1036C00047F0FF0E66EC2BF0000E495CD8B4A2EF79
:1036D0001BF0010E495CD8B4BDEF1BF0020E495C33
:1036E000D8B4D8EF1BF0030E495CD8B4D8EF1BF068
:1036F000040E495CD8B4FFEF1BF0050E495CD8B44A
:103700001AEF1CF0060E495CD8B435EF1CF0CDEC76
:1037100047F0FF0E66EC2BF02DEC48F0FF0E66EC48
:103720002BF00DEC48F0FF0E66EC2BF0FDEC47F0B3
:10373000FF0E66EC2BF0CDEC47F0FF0E66EC2BF0A5
:103740004EEF1CF0DDEC47F0FF0E66EC2BF03DEC8D
:1037500048F0FF0E66EC2BF0BDEC48F0000E66EC76
:103760002BF0BDEC48F0000E66EC2BF0BDEC48F001
:10377000000E66EC2BF04EEF1CF03DEC48F0FF0E17
:1037800066EC2BF06DEC47F0FF0E66EC2BF0BDEC19
:1037900048F0000E66EC2BF0BDEC48F0000E66EC35
:1037A0002BF0BDEC48F0000E66EC2BF04EEF1CF059
:1037B0002DEC48F0FF0E66EC2BF05DEC47F0FF0EB1
:1037C00066EC2BF03DEC48F0FF0E66EC2BF0020EA1
:1037D000495CD8B4F3EF1BF04DEC43F0FF0E66EC00
:1037E0002BF0F8EF1BF05DEC43F0FF0E66EC2BF0D6
:1037F000BDEC48F0000E66EC2BF04EEF1CF0ADEC8B
:1038000047F0FF0E66EC2BF05DEC48F0FF0E66EC27
:103810002BF03DEC48F0FF0E66EC2BF04DEC48F041
:10382000FF0E66EC2BF0BDEC48F0000E66EC2BF0C2
:103830004EEF1CF04DEC47F0FF0E66EC2BF05DEC0C
:1038400047F0FF0E66EC2BF0CDEC47F0FF0E66EC78
:103850002BF0BDEC48F0000E66EC2BF0BDEC48F010
:10386000000E66EC2BF04EEF1CF03DEC48F0FF0E26
:1038700066EC2BF00DEC48F0FF0E66EC2BF0FDEC47
:1038800047F0FF0E66EC2BF0CDEC47F0FF0E66EC38
:103890002BF0BDEC48F0000E66EC2BF03FB655EF78
:1038A0001CF03F8616504A6E4B6E97EC32F02BECB4
:1038B0002BF0400E34EC2BF0BD0E4DEC2BF04050B5
:1038C00044EC3AF08DEC3AF03F82FEEF20F060ECF1
:1038D0003FF03FB26EEF1CF0070E496E3FA45AEC6A
:1038E00032F028EC2BF0460E34EC2BF0BC0E4DECF5
:1038F0002BF0010E495CD8B4C4EF1CF0020E495CF9
:10390000D8B4ECEF1CF0030E495CD8B414EF1DF0F2
:10391000040E495CD8B43CEF1DF0050E495CD8B4E8
:1039200064EF1DF0060E495CD8B48CEF1DF0080E54
:10393000495CD8B4B2EF1DF0FF0E66EC2BF00DEC35
:1039400048F0FF0E66EC2BF01DEC47F0FF0E66EC26
:103950002BF02DEC48F0FF0E66EC2BF0DDEC47F081
:10396000FF0E66EC2BF0BDEC48F0000E66EC2BF081
:10397000BDEC48F0000E66EC2BF0BDEC48F0000EFC
:1039800066EC2BF0B2EF1DF0FF0E66EC2BF01DEC99
:1039900048F0FF0E66EC2BF03DEC47F0FF0E66ECB6
:1039A0002BF02DEC48F0FF0E66EC2BF03DEC47F0D1
:1039B000FF0E66EC2BF0DDEC47F0FF0E66EC2BF013
:1039C000BDEC48F0000E66EC2BF0BDEC48F0000EAC
:1039D00066EC2BF0B2EF1DF0FF0E66EC2BF03DEC29
:1039E00047F0FF0E66EC2BF03DEC47F0FF0E66EC67
:1039F0002BF02DEC48F0FF0E66EC2BF03DEC47F081
:103A0000FF0E66EC2BF0DDEC47F0FF0E66EC2BF0C2
:103A1000BDEC48F0000E66EC2BF0BDEC48F0000E5B
:103A200066EC2BF0B2EF1DF0FF0E66EC2BF05DECB8
:103A300048F0FF0E66EC2BF0EDEC47F0FF0E66EC65
:103A40002BF0CDEC47F0FF0E66EC2BF0FDEC47F0D1
:103A5000FF0E66EC2BF03DEC47F0FF0E66EC2BF012
:103A6000BDEC47F0FF0E66EC2BF0DDEC47F0FF0EEF
:103A700066EC2BF0B2EF1DF0FF0E66EC2BF06DEC58
:103A800048F0FF0E66EC2BF0DDEC47F0FF0E66EC25
:103A90002BF0BDEC48F0000E66EC2BF0BDEC48F0CE
:103AA000000E66EC2BF0BDEC48F0000E66EC2BF03F
:103AB000BDEC48F0000E66EC2BF0BDEC48F0000EBB
:103AC00066EC2BF0B2EF1DF0FF0E66EC2BF03DEC38
:103AD00047F0FF0E66EC2BF0FDEC47F0FF0E66ECB6
:103AE0002BF0DDEC47F0FF0E66EC2BF06DEC47F0B1
:103AF000FF0E66EC2BF0DDEC47F0FF0E66EC2BF0D2
:103B0000BDEC48F0000E66EC2BF0BDEC48F0000E6A
:103B100066EC2BF0B2EF1DF0FF0E66EC2BF02DECF7
:103B200047F0FF0E66EC2BF09DEC47F0FF0E66ECC5
:103B30002BF00DEC48F0FF0E66EC2BF0DDEC47F0BF
:103B4000FF0E66EC2BF0BDEC48F0000E66EC2BF09F
:103B5000BDEC48F0000E66EC2BF0BDEC48F0000E1A
:103B600066EC2BF03FB6B9EF1DF03F8617504A6E5A
:103B70004B6E97EC32F02BEC2BF0400E34EC2BF02C
:103B8000BD0E4DEC2BF0405044EC3AF08DEC3AF089
:103B90003F82FEEF20F0EEEC3FF03FB2D2EF1DF09F
:103BA000070E496E3FA45AEC32F028EC2BF0460E7B
:103BB00034EC2BF0BC0E4DEC2BF0010E495CD8B46C
:103BC00013EF1EF0020E495CD8B421EF1EF0030E75
:103BD000495CD8B42AEF1EF0040E495CD8B438EF23
:103BE0001EF0050E495CD8B44BEF1EF0060E495C82
:103BF000D8B459EF1EF0080E495CD8B46AEF1EF035
:103C0000FAEC41F0DDEC47F0FF0E66EC2BF0BDEC7A
:103C100048F0000E66EC2BF0BDEC48F0000E66ECB0
:103C20002BF06AEF1EF06FEC41F0DDEC47F0FF0E79
:103C300066EC2BF0BDEC48F0000E66EC2BF06AEF62
:103C40001EF087EC41F0DDEC47F0FF0E66EC2BF048
:103C50006AEF1EF0A4EC41F0DDEC47F0FF0E66ECDD
:103C60002BF0BDEC48F0000E66EC2BF06AEF1EF076
:103C7000BCEC41F0DDEC47F0FF0E66EC2BF0BDEC48
:103C800048F0000E66EC2BF0BDEC48F0000E66EC40
:103C90002BF06AEF1EF0CFEC41F0DDEC47F0FF0EA9
:103CA00066EC2BF0BDEC48F0000E66EC2BF06AEFF2
:103CB0001EF0E7EC41F0DDEC47F0FF0E66EC2BF078
:103CC000BDEC48F0000E66EC2BF0BDEC48F0000EA9
:103CD00066EC2BF03FB671EF1EF03F8618504A6E2F
:103CE0004B6E97EC32F02BEC2BF0400E34EC2BF0BB
:103CF000BD0E4DEC2BF0405044EC3AF08DEC3AF018
:103D00003F82FEEF20F05DEC40F03FB28AEF1EF004
:103D1000070E496E3FA45AEC32F028EC2BF0460E09
:103D200034EC2BF0BC0E4DEC2BF0010E495CD8B4FA
:103D3000CBEF1EF0020E495CD8B4D9EF1EF0030E93
:103D4000495CD8B4E2EF1EF0040E495CD8B4F0EF41
:103D50001EF0050E495CD8B403EF1FF0060E495C57
:103D6000D8B411EF1FF0080E495CD8B422EF1FF051
:103D7000FAEC41F05DEC43F0FF0E66EC2BF0BDEC8D
:103D800048F0000E66EC2BF0BDEC48F0000E66EC3F
:103D90002BF022EF1FF06FEC41F05DEC43F0FF0ED3
:103DA00066EC2BF0BDEC48F0000E66EC2BF022EF39
:103DB0001FF087EC41F05DEC43F0FF0E66EC2BF05A
:103DC00022EF1FF0A4EC41F05DEC43F0FF0E66EC37
:103DD0002BF0BDEC48F0000E66EC2BF022EF1FF04C
:103DE000BCEC41F05DEC43F0FF0E66EC2BF0BDEC5B
:103DF00048F0000E66EC2BF0BDEC48F0000E66ECCF
:103E00002BF022EF1FF0CFEC41F05DEC43F0FF0E02
:103E100066EC2BF0BDEC48F0000E66EC2BF022EFC8
:103E20001FF0E7EC41F05DEC43F0FF0E66EC2BF089
:103E3000BDEC48F0000E66EC2BF0BDEC48F0000E37
:103E400066EC2BF03FB629EF1FF03F8619504A6E03
:103E50004B6E97EC32F02BEC2BF0400E34EC2BF049
:103E6000BD0E4DEC2BF0405044EC3AF08DEC3AF0A6
:103E70003F82FEEF20F0E6EC40F03FB242EF1FF051
:103E8000070E496E3FA45AEC32F028EC2BF0460E98
:103E900034EC2BF0BC0E4DEC2BF0010E495CD8B489
:103EA00083EF1FF0020E495CD8B491EF1FF0030EB0
:103EB000495CD8B49AEF1FF0040E495CD8B4A8EF5F
:103EC0001FF0050E495CD8B4BBEF1FF0060E495C2D
:103ED000D8B4C9EF1FF0080E495CD8B4DAEF1FF070
:103EE000FAEC41F04DEC43F0FF0E66EC2BF0BDEC2C
:103EF00048F0000E66EC2BF0BDEC48F0000E66ECCE
:103F00002BF0DAEF1FF06FEC41F04DEC43F0FF0EB9
:103F100066EC2BF0BDEC48F0000E66EC2BF0DAEF0F
:103F20001FF087EC41F04DEC43F0FF0E66EC2BF0F8
:103F3000DAEF1FF0A4EC41F04DEC43F0FF0E66EC1D
:103F40002BF0BDEC48F0000E66EC2BF0DAEF1FF022
:103F5000BCEC41F04DEC43F0FF0E66EC2BF0BDECF9
:103F600048F0000E66EC2BF0BDEC48F0000E66EC5D
:103F70002BF0DAEF1FF0CFEC41F04DEC43F0FF0EE9
:103F800066EC2BF0BDEC48F0000E66EC2BF0DAEF9F
:103F90001FF0E7EC41F04DEC43F0FF0E66EC2BF028
:103FA000BDEC48F0000E66EC2BF0BDEC48F0000EC6
:103FB00066EC2BF03FB6E1EF1FF03F861A504A6ED9
:103FC0004B6E97EC32F02BEC2BF0400E34EC2BF0D8
:103FD000BD0E4DEC2BF0405044EC3AF08DEC3AF035
:103FE0003F82FEEF20F0BDEC45F0000E66EC2BF0BA
:103FF000CDEC45F0000E66EC2BF0DDEC45F0000E4C
:1040000066EC2BF08DEC45F0000E66EC2BF0BDEC71
:1040100046F0000E66EC2BF02DEC46F0000E66EC40
:104020002BF0ADEC46F0000E66EC2BF0BDEC48F04A
:104030002DEC46F0000E66EC2BF05DEC46F02BEC20
:104040002BF0400E34EC2BF0B90E4DEC2BF0000EA3
:1040500066EC2BF08DEC45F0000E66EC2BF0BDEC21
:1040600045F0000E66EC2BF028EC2BF0670E34ECDC
:104070002BF0BC0E4DEC2BF03FB053EF20F0000EB8
:1040800066EC2BF0FDEC46F0000E66EC2BF0CDEC70
:1040900045F0000E66EC2BF09DEC46F0000E66EC51
:1040A0002BF065EF20F0FF0E66EC2BF09DEC48F056
:1040B000FF0E66EC2BF05DEC47F0FF0E66EC2BF08C
:1040C0003DEC48F0FF0E66EC2BF02BEC2BF0440E91
:1040D00034EC2BF0BC0E4DEC2BF03FB084EF20F015
:1040E000FF0E66EC2BF0EDEC47F0FF0E66EC2BF0CC
:1040F000CDEC48F0FF0E66EC2BF0FDEC47F0FF0E28
:1041000066EC2BF096EF20F0000E66EC2BF04DECF9
:1041100046F0000E66EC2BF0BDEC48F0000E66ECAD
:104120002BF05DEC46F0000E66EC2BF080B0AFEFAC
:1041300020F0070E555CD8B4A1EF20F0552AB1EF5E
:1041400020F0556A3EB0B1EF20F03FB0ABEF20F069
:104150003F80ACEF20F03F903E80B1EF20F03E90EA
:10416000556A84B6CAEF20F0070E545CD8B4BCEF91
:1041700020F0542ACCEF20F0546A3EBCCCEF20F063
:104180003FB0C6EF20F03F80C7EF20F03F903E8C5D
:10419000CCEF20F03E9C546A80B8FCEF20F0070E74
:1041A000575CD8B4D7EF20F0572AFEEF20F0576ABB
:1041B0003EB8FEEF20F0436A466A50EC2CF03FA078
:1041C000F8EF20F0080E116E040E126E4B0E136EF7
:1041D000BB0E146E9B0E156E880E166E7F0E176E3C
:1041E0007F0E186E000E196E000E1A6E6DEC2CF01C
:1041F0003F903E8823EF01F03E98576A3FB41FEF8F
:1042000021F080BA1DEF21F0070E565CD8B40CEFF8
:1042100021F0562A1FEF21F0566A3EBA23EF01F033
:10422000000E436E3E8A466A50EC2CF03F903F925F
:104230003F96496A4A6A23EF01F03E9A566A23EF95
:1042400001F028EC2BF0410E34EC2BF0B80E4DECC5
:104250002BF0700E66EC2BF0100E66EC2BF0100EAF
:1042600066EC2BF0100E66EC2BF0000E66EC2BF0DB
:10427000CDEC45F0000E66EC2BF0CDEC45F0000ED9
:1042800066EC2BF06DEC46F0000E66EC2BF08DEC3E
:1042900046F0000E66EC2BF05DEC46F0000E66EC8E
:1042A0002BF03DEC46F0000E66EC2BF0BDEC48F038
:1042B000DDEC46F0000E66EC2BF08DEC46F0000EC7
:1042C00066EC2BF00DEC46F02BEC2BF0400E34ECB2
:1042D0002BF0B80E4DEC2BF0000E66EC2BF0ADEC95
:1042E00046F0000E66EC2BF0CDEC45F0000E66ECCF
:1042F0002BF0082A320E085CD8B484EF21F0100E9F
:1043000066EC2BF079EF21F0086A700E66EC2BF06A
:10431000000E445CD8B494EF21F0010E445CD8B494
:104320003CEF25F023EF01F028EC2BF0460E34ECA7
:104330002BF0B90E4DEC2BF09DEC46F0000E66EC28
:104340002BF0CDEC45F0000E66EC2BF02DEC46F09A
:10435000000E66EC2BF0CDEC45F0000E66EC2BF079
:10436000ADEC45F0000E66EC2BF0ADEC46F0000E27
:1043700066EC2BF0BDEC48F08DEC45F0000E66ECE1
:104380002BF0BDEC45F0000E66EC2BF0BDEC45F0DB
:104390002BEC2BF0400E34EC2BF0B90E4DEC2BF047
:1043A000000E66EC2BF08DEC46F0000E66EC2BF068
:1043B000CDEC45F0000E66EC2BF09DEC46F0000EC7
:1043C00066EC2BF09DEC46F0000E66EC2BF080B016
:1043D00002EF22F0070E555CD8B4F2EF21F0552A17
:1043E00004EF22F0556A3EB004EF22F00B0E475C5A
:1043F000D8B4FEEF21F0472AFFEF21F0476A3E8054
:1044000004EF22F03E90556A84B620EF22F0070EAA
:10441000545CD8B40FEF22F0542A22EF22F0546AF1
:104420003EBC22EF22F0000E475CD8B41BEF22F016
:1044300047061DEF22F00B0E476E3E8C22EF22F056
:104440003E9C546A28EC2BF04A0E34EC2BF0BB0E49
:104450004DEC2BF0000E475CD8B443EF22F0000E79
:1044600066EC2BF0ADEC42F0000E66EC2BF0ADEC00
:1044700042F0000E66EC2BF0FDEC45F0000E66EC11
:104480002BF055EF22F0FF0E66EC2BF04DEC43F0D5
:10449000FF0E66EC2BF04DEC43F0FF0E66EC2BF0BC
:1044A0008DEC47F0FF0E66EC2BF028EC2BF0670E3E
:1044B00034EC2BF0BB0E4DEC2BF0010E475CD8B466
:1044C00076EF22F0000E66EC2BF0ADEC42F0000E21
:1044D00066EC2BF0BDEC42F0000E66EC2BF0FDEC30
:1044E00045F0000E66EC2BF088EF22F0FF0E66EC34
:1044F0002BF04DEC43F0FF0E66EC2BF05DEC43F03F
:10450000FF0E66EC2BF08DEC47F0FF0E66EC2BF007
:104510002BEC2BF0440E34EC2BF0BB0E4DEC2BF0BF
:10452000020E475CD8B4A9EF22F0000E66EC2BF027
:10453000ADEC42F0000E66EC2BF0CDEC42F0000E3C
:1045400066EC2BF0FDEC45F0000E66EC2BF0BBEFBB
:1045500022F0FF0E66EC2BF04DEC43F0FF0E66EC04
:104560002BF06DEC43F0FF0E66EC2BF08DEC47F07A
:10457000FF0E66EC2BF02BEC2BF0610E34EC2BF0E5
:10458000BB0E4DEC2BF0030E475CD8B4DCEF22F0F1
:10459000000E66EC2BF0ADEC42F0000E66EC2BF05A
:1045A000DDEC42F0000E66EC2BF0FDEC45F0000E69
:1045B00066EC2BF0EEEF22F0FF0E66EC2BF04DECEC
:1045C00043F0FF0E66EC2BF07DEC43F0FF0E66EC43
:1045D0002BF08DEC47F0FF0E66EC2BF028EC2BF067
:1045E0004A0E34EC2BF0BC0E4DEC2BF0040E475C65
:1045F000D8B40FEF23F0000E66EC2BF0ADEC42F0D8
:10460000000E66EC2BF0EDEC42F0000E66EC2BF0A9
:10461000FDEC45F0000E66EC2BF021EF23F0FF0ED1
:1046200066EC2BF04DEC43F0FF0E66EC2BF08DECBE
:1046300043F0FF0E66EC2BF08DEC47F0FF0E66ECBE
:104640002BF028EC2BF0670E34EC2BF0BC0E4DEC6D
:104650002BF0050E475CD8B442EF23F0000E66EC59
:104660002BF0ADEC42F0000E66EC2BF0FDEC42F0CE
:10467000000E66EC2BF0FDEC45F0000E66EC2BF026
:1046800054EF23F0FF0E66EC2BF04DEC43F0FF0EE1
:1046900066EC2BF09DEC43F0FF0E66EC2BF08DECFE
:1046A00047F0FF0E66EC2BF02BEC2BF0440E34ECB5
:1046B0002BF0BC0E4DEC2BF0060E475CD8B475EF1A
:1046C00023F0000E66EC2BF0ADEC42F0000E66EC31
:1046D0002BF00DEC43F0000E66EC2BF0FDEC45F0FA
:1046E000000E66EC2BF087EF23F0FF0E66EC2BF04C
:1046F0004DEC43F0FF0E66EC2BF0ADEC43F0FF0EFB
:1047000066EC2BF08DEC47F0FF0E66EC2BF02BECFB
:104710002BF0610E34EC2BF0B40E4DEC2BF0070EA9
:10472000475CD8B4A8EF23F0000E66EC2BF0ADEC9C
:1047300042F0000E66EC2BF01DEC43F0000E66EC30
:104740002BF0FDEC45F0000E66EC2BF0BAEF23F0F9
:10475000FF0E66EC2BF04DEC43F0FF0E66EC2BF0F9
:10476000BDEC43F0FF0E66EC2BF08DEC47F0FF0E36
:1047700066EC2BF028EC2BF04A0E34EC2BF0BD0E3F
:104780004DEC2BF0080E475CD8B4DBEF23F0000EA5
:1047900066EC2BF0ADEC42F0000E66EC2BF02DEC4D
:1047A00043F0000E66EC2BF0FDEC45F0000E66ECDD
:1047B0002BF0EDEF23F0FF0E66EC2BF04DEC43F009
:1047C000FF0E66EC2BF0CDEC43F0FF0E66EC2BF009
:1047D0008DEC47F0FF0E66EC2BF028EC2BF0670E0B
:1047E00034EC2BF0BD0E4DEC2BF0090E475CD8B429
:1047F0000EEF24F0000E66EC2BF0ADEC42F0000E54
:1048000066EC2BF03DEC43F0000E66EC2BF0FDEC7B
:1048100045F0000E66EC2BF020EF24F0FF0E66EC66
:104820002BF04DEC43F0FF0E66EC2BF0DDEC43F08B
:10483000FF0E66EC2BF08DEC47F0FF0E66EC2BF0D4
:1048400028EC2BF04A0E34EC2BF0BE0E4DEC2BF086
:104850000A0E475CD8B45CEF24F0000E66EC2BF037
:104860005DEC46F0000E66EC2BF0ADEC46F0000E71
:1048700066EC2BF0FDEC45F0000E66EC2BF0CDEC79
:1048800045F0000E66EC2BF08DEC46F0000E66EC69
:104890002BF0BDEC48F09DEC46F0000E66EC2BF0E2
:1048A000CDEC45F0000E66EC2BF0ADEC46F0000EC2
:1048B00066EC2BF089EF24F0FF0E66EC2BF0FDEC9C
:1048C00047F0FF0E66EC2BF04DEC48F0FF0E66EC67
:1048D0002BF08DEC47F0FF0E66EC2BF05DEC47F013
:1048E000FF0E66EC2BF02DEC48F0FF0E66EC2BF083
:1048F000CDEC48F03DEC48F0FF0E66EC2BF05DECA3
:1049000047F0FF0E66EC2BF04DEC48F0FF0E66EC26
:104910002BF028EC2BF04A0E34EC2BF0BF0E4DECB4
:104920002BF00B0E475CD8B4DCEF24F0000E66ECE5
:104930002BF08DEC45F0000E66EC2BF02DEC46F0E4
:10494000000E66EC2BF02DEC46F0000E66EC2BF022
:10495000BDEC48F08DEC46F0000E66EC2BF0CDEC93
:1049600045F0000E66EC2BF0EDEC45F0000E66EC29
:104970002BF00DEC46F0000E66EC2BF09DEC46F0B3
:10498000000E66EC2BF02BEC2BF0400E34EC2BF0F1
:10499000BF0E4DEC2BF0ADEC46F0000E66EC2BF0AC
:1049A000CDEC45F0000E66EC2BF08DEC46F0000EE1
:1049B00066EC2BF020EF25F0FF0E66EC2BF01DECE3
:1049C00047F0FF0E66EC2BF0CDEC47F0FF0E66ECE7
:1049D0002BF0CDEC47F0FF0E66EC2BF0CDEC48F061
:1049E0002DEC48F0FF0E66EC2BF05DEC47F0FF0E6F
:1049F00066EC2BF07DEC47F0FF0E66EC2BF09DECA7
:104A000047F0FF0E66EC2BF03DEC48F0FF0E66EC35
:104A10002BF02BEC2BF0400E34EC2BF0BF0E4DECBA
:104A20002BF04DEC48F0FF0E66EC2BF05DEC47F000
:104A3000FF0E66EC2BF02DEC48F0FF0E66EC2BF031
:104A4000E9EC2EF080B838EF25F0070E575CD8B4AB
:104A50002DEF25F0572A3AEF25F0576A3EB83AEF86
:104A600025F0010E446E50EC2CF03E883AEF25F014
:104A70003E98576A23EF01F028EC2BF0460E34ECF9
:104A80002BF0B90E4DEC2BF0000E475CD8B47DEF47
:104A900025F0010E475CD8B485EF25F0020E475C87
:104AA000D8B48DEF25F0030E475CD8B495EF25F010
:104AB000040E475CD8B49DEF25F0050E475CD8B4D2
:104AC000A5EF25F0060E475CD8B4ADEF25F0070E34
:104AD000475CD8B4B5EF25F0080E475CD8B4BDEFFD
:104AE00025F0090E475CD8B4C5EF25F00A0E475CE7
:104AF000D8B4CDEF25F027EF26F0FAEC3CF02BEC04
:104B000035F0C4EC35F0B8EF26F053EC3DF02BEC6B
:104B100035F0C4EC35F0B8EF26F0ACEC3DF02BEC02
:104B200035F0C4EC35F0B8EF26F005EC3EF02BEC98
:104B300035F0C4EC35F0B8EF26F05EEC3EF02BEC2F
:104B400035F0C4EC35F0B8EF26F0B7EC3EF02BECC6
:104B500035F0C4EC35F0B8EF26F060EC3FF02BEC0C
:104B600035F0C4EC35F0B8EF26F0EEEC3FF02BEC6E
:104B700035F0C4EC35F0B8EF26F05DEC40F02BECEE
:104B800035F0C4EC35F0B8EF26F0E6EC40F02BEC55
:104B900035F0C4EC35F0B8EF26F0000E66EC2BF0E3
:104BA0005DEC46F0000E66EC2BF0ADEC46F0000E2E
:104BB00066EC2BF0FDEC45F0000E66EC2BF0CDEC36
:104BC00045F0000E66EC2BF08DEC46F0000E66EC26
:104BD0002BF0BDEC48F09DEC46F0000E66EC2BF09F
:104BE000CDEC45F0000E66EC2BF0ADEC46F0000E7F
:104BF00066EC2BF02BEC2BF0400E34EC2BF0B90EC6
:104C00004DEC2BF0000E66EC2BF0000E66EC2BF05A
:104C1000DDEC46F0000E66EC2BF08DEC46F0000E5D
:104C200066EC2BF00DEC46F0000E66EC2BF0ADECD4
:104C300046F0000E66EC2BF0CDEC45F0000E66EC75
:104C40002BF02BEC35F0C4EC35F0B8EF26F08DEC02
:104C500045F0000E66EC2BF02DEC46F0000E66ECF5
:104C60002BF02DEC46F0000E66EC2BF0BDEC48F07E
:104C70008DEC46F0000E66EC2BF0CDEC45F0000E0E
:104C800066EC2BF0EDEC45F0000E66EC2BF00DEC35
:104C900046F0000E66EC2BF09DEC46F0000E66EC44
:104CA0002BF0ADEC46F02BEC2BF0400E34EC2BF05F
:104CB000B90E4DEC2BF0000E66EC2BF0CDEC45F070
:104CC000000E66EC2BF08DEC46F0000E66EC2BF03F
:104CD000BDEC48F0DDEC46F0000E66EC2BF08DEC00
:104CE00046F0000E66EC2BF00DEC46F0000E66EC84
:104CF0002BF0ADEC46F0000E66EC2BF0CDEC45F061
:104D0000000E66EC2BF02BEC35F080B8B6EF26F0F9
:104D1000070E575CD8B490EF26F0572AB8EF26F06C
:104D2000576A3EB8B8EF26F03FACAFEF26F050EC34
:104D30002CF0F5EC48F008EC49F01BEC49F02EECB7
:104D400049F041EC49F054EC49F067EC49F07AEC59
:104D500049F08DEC49F0A0EC49F0B3EC49F0446A1D
:104D6000476A3F9C3F903E8823EF01F03E98576A88
:104D700080BA23EF01F0070E565CD8B4C3EF26F0DB
:104D8000562A23EF01F0566A000E446E3E8A476AA7
:104D900050EC2CF03F9C23EF01F028EC2BF0410E5F
:104DA00034EC2BF0B80E4DEC2BF0700E66EC2BF0C3
:104DB000100E66EC2BF0100E66EC2BF0100E66EC6D
:104DC0002BF0000E66EC2BF05DEC46F0000E66EC6E
:104DD0002BF0ADEC46F0000E66EC2BF0FDEC45F050
:104DE000000E66EC2BF0CDEC45F0000E66EC2BF0DF
:104DF0008DEC46F0000E66EC2BF0BDEC48F09DEC1F
:104E000046F0000E66EC2BF0CDEC45F0000E66ECA3
:104E10002BF0ADEC46F0000E66EC2BF0ADEC46F05E
:104E20002BEC2BF0400E34EC2BF0B80E4DEC2BF0AD
:104E3000000E66EC2BF00DEC46F0000E66EC2BF04D
:104E40004DEC46F0000E66EC2BF0EDEC45F0000E5C
:104E500066EC2BF0082A2C0E085CD8B435EF27F04E
:104E6000100E66EC2BF02AEF27F0086A700E66EC45
:104E70002BF028EC2BF0460E34EC2BF0BF0E4DEC53
:104E80002BF09DEC46F0000E66EC2BF05DEC46F04E
:104E9000000E66EC2BF0DDEC45F0000E66EC2BF01E
:104EA000ADEC46F0000E66EC2BF0DDEC46F0000EAB
:104EB00066EC2BF08DEC45F0000E66EC2BF08DECE3
:104EC00046F0000E66EC2BF0CDEC45F0000E66ECE3
:104ED0002BF0BDEC48F0CDEC46F02BEC2BF0400E67
:104EE00034EC2BF0BF0E4DEC2BF0000E66EC2BF0EB
:104EF000CDEC45F0000E66EC2BF08DEC46F0000E8C
:104F000066EC2BF09DEC46F0000E66EC2BF00DEC01
:104F100046F0000E66EC2BF05DEC46F0000E66EC01
:104F20002BF04DEC46F0000E66EC2BF0BDEC48F09B
:104F3000000E66EC2BF0BDEC42F0000E66EC2BF0A0
:104F4000000E66EC2BF0400E66EC2BF0000E66ECCB
:104F50002BF0ADEC42F0000E66EC2BF0CDEC42F005
:104F6000000E66EC2BF028EC2BF0450E34EC2BF009
:104F7000BA0E4DEC2BF04CBEFFEF27F0000E485C54
:104F8000D8A4FFEF27F0FF0E66EC2BF05DEC47F0A6
:104F9000FF0E66EC2BF02DEC48F0FF0E66EC2BF0CC
:104FA0002DEC48F0FF0E66EC2BF0FDEC47F0FF0E09
:104FB00066EC2BF02DEC48F0FF0E66EC2BF0CDEC00
:104FC00048F08DEC47F0FF0E66EC2BF0FDEC47F05F
:104FD000FF0E66EC2BF0CDEC47F0FF0E66EC2BF0ED
:104FE0004DEC47F02BEC2BF0400E34EC2BF0BA0ECE
:104FF0004DEC2BF0FF0E66EC2BF039EF28F0000E95
:1050000066EC2BF0CDEC45F0000E66EC2BF08DEC51
:1050100046F0000E66EC2BF08DEC46F0000E66ECD0
:105020002BF05DEC46F0000E66EC2BF08DEC46F0BC
:10503000000E66EC2BF0BDEC48F0FDEC45F0000EE8
:1050400066EC2BF05DEC46F0000E66EC2BF02DECE0
:1050500046F0000E66EC2BF0BDEC45F02BEC2BF08F
:10506000400E34EC2BF0BA0E4DEC2BF0000E66EC3B
:105070002BF028EC2BF0450E34EC2BF0BB0E4DEC56
:105080002BF04CBE78EF28F0010E485CD8A478EFE6
:1050900028F0FF0E66EC2BF04DEC48F0FF0E66ECAE
:1050A0002BF08DEC48F0FF0E66EC2BF0CDEC48F0C9
:1050B000FDEC47F0FF0E66EC2BF05DEC48F0FF0EC8
:1050C00066EC2BF04DEC48F0FF0E66EC2BF00DEC8F
:1050D00048F0FF0E66EC2BF05DEC48F0FF0E66EC3E
:1050E0002BF04DEC48F0FF0E66EC2BF0A5EF28F00E
:1050F000000E66EC2BF0ADEC46F0000E66EC2BF0EB
:10510000EDEC46F0000E66EC2BF0BDEC48F05DECEB
:1051100046F0000E66EC2BF0BDEC46F0000E66EC9F
:105120002BF0ADEC46F0000E66EC2BF06DEC46F08B
:10513000000E66EC2BF0BDEC46F0000E66EC2BF09A
:10514000ADEC46F0000E66EC2BF028EC2BF0450E93
:1051500034EC2BF0BC0E4DEC2BF04CBEF1EF28F0F4
:10516000020E485CD8A4F1EF28F0FF0E66EC2BF09D
:105170003DEC48F0FF0E66EC2BF05DEC47F0FF0EC7
:1051800066EC2BF0CDEC47F0FF0E66EC2BF05DECFF
:1051900047F0FF0E66EC2BF03DEC47F0FF0E66EC9F
:1051A0002BF04DEC48F0FF0E66EC2BF0CDEC48F008
:1051B0005DEC48F0FF0E66EC2BF03DEC48F0FF0E86
:1051C00066EC2BF02DEC47F02BEC2BF0400E34EC82
:1051D0002BF0BC0E4DEC2BF0FF0E66EC2BF02BEF02
:1051E00029F0000E66EC2BF09DEC46F0000E66EC0C
:1051F0002BF0CDEC45F0000E66EC2BF02DEC46F0DC
:10520000000E66EC2BF0CDEC45F0000E66EC2BF0BA
:10521000ADEC45F0000E66EC2BF0ADEC46F0000E68
:1052200066EC2BF0BDEC48F0BDEC46F0000E66ECF1
:105230002BF09DEC46F0000E66EC2BF09DEC45F05B
:105240002BEC2BF0400E34EC2BF0BC0E4DEC2BF085
:10525000000E66EC2BF04CBE69EF29F080B049EFF0
:1052600029F0070E555CD8B439EF29F0552A4BEFD9
:1052700029F0556A3EB04BEF29F0020E485CD8B4D5
:1052800045EF29F0482A46EF29F0486A3E804BEF67
:1052900029F03E90556A84B667EF29F0070E545CFA
:1052A000D8B456EF29F0542A69EF29F0546A3EBC6D
:1052B00069EF29F0000E485CD8B462EF29F0480687
:1052C00064EF29F0020E486E3E8C69EF29F03E9C97
:1052D000546A4CBE83EF29F080B881EF29F0070EA5
:1052E000575CD8B477EF29F0572A83EF29F0576A33
:1052F0003EB883EF29F04C8E4C504D6E3E8883EFC4
:1053000029F03E98576A4CAE9DEF29F080BA9BEF8A
:1053100029F0070E565CD8B491EF29F0562A9DEF7C
:1053200029F0566A3EBA9DEF29F04C9E50EC2CF0C5
:105330003E8A9DEF29F03E9A566A4CAEB9EF29F0AD
:1053400080B8B7EF29F0070E575CD8B4ABEF29F05F
:10535000572AB9EF29F0576A3EB8B9EF29F04D50F6
:105360004C6E4C9E50EC2CF03E88B9EF29F03E98E4
:10537000576A4CAE14EF2AF080B0E6EF29F0070E22
:10538000555CD8B4C7EF29F0552AE8EF29F0556AE3
:105390003EB0E8EF29F0000E485CD8B4DCEF29F00D
:1053A000010E485CD8B4DFEF29F0020E485CD8B497
:1053B000E2EF29F0E3EF29F04D70E3EF29F04D72B1
:1053C000E3EF29F04D743E80E8EF29F03E90556AF6
:1053D00084B612EF2AF0070E545CD8B4F3EF29F02C
:1053E000542A14EF2AF0546A3EBC14EF2AF0000E3F
:1053F000485CD8B408EF2AF0010E485CD8B40BEF33
:105400002AF0020E485CD8B40EEF2AF00FEF2AF013
:105410004D700FEF2AF04D720FEF2AF04D743E8C55
:1054200014EF2AF03E9C546A4CAE23EF2BF0000E92
:10543000485CD8B428EF2AF0010E485CD8B465EF78
:105440002AF0020E485CD8B4D4EF2AF023EF2BF0F8
:105450002BEC2BF0460E34EC2BF0BA0E4DEC2BF06F
:105460004DA04CEF2AF0FF0E66EC2BF08DEC47F0D0
:10547000FF0E66EC2BF0FDEC47F0FF0E66EC2BF018
:10548000CDEC47F0FF0E66EC2BF04DEC47F0FF0E35
:1054900066EC2BF023EF2BF0FF0E66EC2BF06DEC9F
:1054A00047F0FF0E66EC2BF02DEC48F0FF0E66EC9B
:1054B0002BF05DEC47F0FF0E66EC2BF05DEC47F057
:1054C000FF0E66EC2BF023EF2BF02BEC2BF0460EAF
:1054D00034EC2BF0BB0E4DEC2BF04DA2A2EF2AF0DA
:1054E000FF0E66EC2BF09DEC47F0FF0E66EC2BF008
:1054F000EDEC47F0FF0E66EC2BF04DEC48F0FF0EA4
:1055000066EC2BF05DEC47F0FF0E66EC2BF02DEC1B
:1055100048F0FF0E66EC2BF0CDEC47F0FF0E66EC8A
:105520002BF0FDEC47F0FF0E66EC2BF03DEC47F066
:10553000FF0E66EC2BF0BDEC47F0FF0E66EC2BF097
:1055400023EF2BF0FF0E66EC2BF06DEC47F0FF0E17
:1055500066EC2BF02DEC48F0FF0E66EC2BF05DECCA
:1055600047F0FF0E66EC2BF05DEC47F0FF0E66ECAB
:105570002BF0BDEC48F0000E66EC2BF0BDEC48F0D3
:10558000000E66EC2BF0BDEC48F0000E66EC2BF044
:10559000BDEC48F0000E66EC2BF0BDEC48F0000EC0
:1055A00066EC2BF023EF2BF02BEC2BF0460E34ECBB
:1055B0002BF0BC0E4DEC2BF04DA402EF2BF0FF0EA8
:1055C00066EC2BF01DEC47F0FF0E66EC2BF05DEC6B
:1055D00048F0FF0E66EC2BF04DEC48F0FF0E66EC49
:1055E0002BF0FDEC47F0FF0E66EC2BF0BDEC48F025
:1055F000000E66EC2BF0BDEC48F0000E66EC2BF0D4
:1056000023EF2BF0FF0E66EC2BF0DDEC47F0FF0EE6
:1056100066EC2BF01DEC47F0FF0E66EC2BF0EDEC8A
:1056200047F0FF0E66EC2BF05DEC48F0FF0E66ECE9
:105630002BF01DEC47F0FF0E66EC2BF0CDEC47F0A5
:10564000FF0E66EC2BF04CAEE9EC2EF023EF01F0F0
:105650008C888B9E12008C988B8E12008C888B8E7F
:1056600012008C988B9E1200016E2DEC2CF00150D4
:105670008A6E8C9C8C9E000000008C8A00000000CA
:105680000000000000000000000000008C9A0000F4
:1056900000000000000000001200026E2DEC2CF053
:1056A00002508A6E8C9C8C9E000000008C8A000048
:1056B00000000000000000000000000000008C9AC4
:1056C000000000000000000000001200006E2DEC41
:1056D0002CF03FBE82EC2BF000508A6E8C9C8C8E9E
:1056E000000000008C8A00000000000000000000A4
:1056F0000000000000008C9A000000000000000084
:1057000000001200000E515CD8B4A7EF2BF0010E80
:10571000515CD8B4C0EF2BF0020E515CD8B4D7EF77
:105720002BF0030E515CD8B4ECEF2BF0040E515C5F
:10573000D8B4FFEF2BF0050E515CD8B410EF2CF06D
:10574000060E515CD8B41FEF2CF02CEF2CF050B0AB
:10575000B5EF2BF0004200420042004200420042FE
:105760000042010E00162CEF2CF0004600460046C9
:105770000046004600460046800E00162CEF2CF036
:1057800050B0CDEF2BF000420042004200420042F8
:105790000042030E00162CEF2CF000460046004697
:1057A000004600460046C00E00162CEF2CF050B00C
:1057B000E3EF2BF000420042004200420042070E9D
:1057C00000162CEF2CF0004600460046004600462E
:1057D000E00E00162CEF2CF050B0F7EF2BF000424B
:1057E0000042004200420F0E00162CEF2CF0004643
:1057F000004600460046F00E00162CEF2CF050B08C
:1058000009EF2CF00042004200421F0E00162CEF60
:105810002CF0004600460046F80E00162CEF2CF047
:1058200050B019EF2CF0004200423F0E00162CEF52
:105830002CF000460046FC0E00162CEF2CF050B069
:1058400027EF2CF000427F0E00162CEF2CF00046C4
:10585000FE0E00162CEF2CF012000F01FF0E936EBF
:1058600000018C8C8C9E000000008C8A00000000DF
:105870000000000000000000000000008C9A000002
:10588000000000000000000000000000000081BED9
:1058900035EF2CF08C9C0F01000E936E000112006E
:1058A0002EEC2BF0400E34EC2BF0B80E4DEC2BF020
:1058B000000E66EC2BF0012A800E015CD8A458EF94
:1058C0002CF0022A4EEC2BF0400E34EC2BF0C00EE4
:1058D000025CD8A458EF2CF012008B8000008B9251
:1058E00076EC37F08B8276EC37F08AEC2CF0A0EC7B
:1058F0002CF0B5EC2CF0CAEC2CF0DFEC2CF0F4EC36
:105900002CF009EC2DF01EEC2DF033EC2DF048ECD2
:105910002DF012008B9000005DEC2DF08B940000B8
:105920008B8600008B960000000E386E88EC2DF000
:1059300011503C6E9DEC2DF08B948B968B80120059
:105940008B905DEC2DF08B9400008B8600008B9685
:105950000000010E386E88EC2DF012503C6E9DEC6C
:105960002DF08B948B968B8012008B905DEC2DF03C
:105970008B9400008B8600008B960000020E386E20
:1059800088EC2DF013503C6E9DEC2DF08B948B9693
:105990008B8012008B905DEC2DF08B9400008B8639
:1059A00000008B960000030E386E88EC2DF014502A
:1059B0003C6E9DEC2DF08B948B968B8012008B901F
:1059C0005DEC2DF08B9400008B8600008B96000020
:1059D000040E386E88EC2DF015503C6E9DEC2DF0C9
:1059E0008B948B968B8012008B905DEC2DF08B94BA
:1059F00000008B8600008B960000050E386E88EC48
:105A00002DF016503C6E9DEC2DF08B948B968B8078
:105A100012008B905DEC2DF08B9400008B860000C3
:105A20008B960000060E386E88EC2DF017503C6EF9
:105A30009DEC2DF08B948B968B8012008B905DECFF
:105A40002DF08B9400008B8600008B960000070ED3
:105A5000386E88EC2DF018503C6E9DEC2DF08B9438
:105A60008B968B8012008B905DEC2DF08B94000058
:105A70008B8600008B960000080E386E88EC2DF0A7
:105A800019503C6E9DEC2DF08B948B968B80120000
:105A90008B905DEC2DF08B9400008B8600008B9634
:105AA0000000090E386E88EC2DF01A503C6E9DEC0B
:105AB0002DF08B948B968B8012008B9400008B863C
:105AC00000008B9600008B9400008B8600008B9664
:105AD00000008B8400008B8600008B9600008B9466
:105AE00000008B8600008B9600008B9400008B8654
:105AF00000008B9600008B9400008B8600008B9634
:105B000000008B9400008B8600008B960000120032
:105B100038BE8EEF2DF08B9490EF2DF08B8400002B
:105B20008B8600008B960000392A3846080E395CB7
:105B3000D8A488EF2DF0396A12003CBEA3EF2DF0F7
:105B40008B94A5EF2DF08B8400008B8600008B9644
:105B500000003A2A3C46080E3A5CD8A49DEF2DF08E
:105B60003A6A12008B905DEC2DF08B9400008B86CE
:105B700000008B9600000A0E386E88EC2DF08B80AA
:105B80000000000000008B905DEC2DF08B84000085
:105B90008B8600008B960000000000000000D5EC12
:105BA0002DF08B948B968B8012008B8683A0DCEF7C
:105BB0002DF03B80DDEF2DF03B903A2A8B96080EBE
:105BC0003A5CD8B4E7EF2DF03B46D5EF2DF03A6ABA
:105BD0003D2A010E3D5CD8A4F2EF2DF03B501B6E28
:105BE000D5EF2DF0020E3D5CD8A4FBEF2DF03B501D
:105BF0001C6ED5EF2DF0030E3D5CD8A404EF2EF003
:105C00003B501D6ED5EF2DF0040E3D5CD8A40DEF7A
:105C10002EF03B501E6ED5EF2DF0050E3D5CD8A446
:105C200016EF2EF03B501F6ED5EF2DF0060E3D5CAB
:105C3000D8A41FEF2EF03B50206ED5EF2DF0070EAD
:105C40003D5CD8A428EF2EF03B50216ED5EF2DF00F
:105C5000080E3D5CD8A431EF2EF03B50226ED5EFFC
:105C60002DF0090E3D5CD8A43AEF2EF03B50236E88
:105C7000D5EF2DF00A0E3D5CD8A443EF2EF03B503B
:105C8000246ED5EF2DF00B0E3D5CD8A44CEF2EF01A
:105C90003B50256ED5EF2DF00C0E3D5CD8A455EF92
:105CA0002EF03B50266ED5EF2DF00D0E3D5CD8A4A6
:105CB0005EEF2EF03B50276ED5EF2DF00E0E3D5CC3
:105CC000D8A467EF2EF03B50286ED5EF2DF00F0EC5
:105CD0003D5CD8A470EF2EF03B50296ED5EF2DF02F
:105CE000100E3D5CD8A479EF2EF03B502A6ED5EF14
:105CF0002DF0110E3D5CD8A482EF2EF03B502B6EA0
:105D0000D5EF2DF0120E3D5CD8A48BEF2EF03B505A
:105D10002C6ED5EF2DF0130E3D5CD8A494EF2EF031
:105D20003B502D6ED5EF2DF0140E3D5CD8A49DEFA9
:105D30002EF03B502E6ED5EF2DF0150E3D5CD8A405
:105D4000A6EF2EF03B502F6ED5EF2DF0160E3D5CDA
:105D5000D8A4AFEF2EF03B50306ED5EF2DF0170EDC
:105D60003D5CD8A4B8EF2EF03B50316ED5EF2DF04E
:105D7000180E3D5CD8A4C1EF2EF03B50326ED5EF2B
:105D80002DF0190E3D5CD8A4CAEF2EF03B50336EB7
:105D9000D5EF2DF01A0E3D5CD8A4D3EF2EF03B507A
:105DA000346ED5EF2DF01B0E3D5CD8A4DCEF2EF049
:105DB0003B50356ED5EF2DF01C0E3D5CD8A4E5EFC1
:105DC0002EF03B50366ED5EF2DF03B50376E3D6ACE
:105DD000120080BAFFEF2EF0070E565CD8B4F4EF35
:105DE0002EF0562A01EF2FF0566A3EBA120050EC00
:105DF0002CF0416A466A476A486A3E8A12003E9A17
:105E0000566A1200000E405CD8A42BEF2FF0EDEC88
:105E100045F0000E66EC2BF04DEC46F0000E66EC03
:105E20002BF0BDEC45F0000E66EC2BF0BDEC48F01D
:105E3000000E66EC2BF0BDEC48F0000E66EC2BF08B
:105E4000BDEC48F0000E66EC2BF0BDEC48F0000E07
:105E500066EC2BF01200010E405CD8A454EF2FF03A
:105E6000CDEC45F0000E66EC2BF03DEC46F0000E5C
:105E700066EC2BF06DEC46F0000E66EC2BF0FDECC2
:105E800045F0000E66EC2BF0BDEC48F0000E66EC21
:105E90002BF0BDEC48F0000E66EC2BF0BDEC48F0AA
:105EA000000E66EC2BF01200020E405CD8A47DEFD1
:105EB0002FF00DEC46F0000E66EC2BF04DEC46F0AA
:105EC000000E66EC2BF0ADEC46F0000E66EC2BF00D
:105ED000BDEC48F0000E66EC2BF0BDEC48F0000E77
:105EE00066EC2BF0BDEC48F0000E66EC2BF0BDEC40
:105EF00048F0000E66EC2BF01200030E405CD8A4B4
:105F0000A6EF2FF0ADEC45F0000E66EC2BF0BDECEB
:105F100048F0000E66EC2BF09DEC46F0000E66ECAF
:105F20002BF0ADEC46F0000E66EC2BF08DEC45F05E
:105F3000000E66EC2BF0BDEC48F0000E66EC2BF08A
:105F4000BDEC48F0000E66EC2BF01200040E405C35
:105F5000D8A4CFEF2FF0BDEC46F0000E66EC2BF08E
:105F6000BDEC48F0000E66EC2BF0BDEC45F0000EE9
:105F700066EC2BF08DEC45F0000E66EC2BF0ADECF2
:105F800046F0000E66EC2BF08DEC45F0000E66EC52
:105F90002BF0BDEC48F0000E66EC2BF01200050E65
:105FA000405CD8A4F8EF2FF08DEC46F0000E66ECC4
:105FB0002BF0BDEC48F0000E66EC2BF0CDEC45F07C
:105FC000000E66EC2BF08DEC46F0000E66EC2BF02C
:105FD0008DEC46F0000E66EC2BF0BDEC48F0000EA8
:105FE00066EC2BF0BDEC48F0000E66EC2BF01200D6
:105FF000060E405CD8A421EF30F04DEC46F0000EC8
:1060000066EC2BF0CDEC46F0000E66EC2BF0BDEC10
:1060100048F0000E66EC2BF0CDEC45F0000E66EC7F
:106020002BF08DEC46F0000E66EC2BF08DEC46F07C
:10603000000E66EC2BF0BDEC48F0000E66EC2BF089
:106040001200070E405CD8A44AEF30F08DEC46F009
:10605000000E66EC2BF0ADEC45F0000E66EC2BF07C
:106060009DEC45F0000E66EC2BF02DEC46F0000E9A
:1060700066EC2BF0BDEC48F0000E66EC2BF0BDECAE
:1060800048F0000E66EC2BF0BDEC48F0000E66EC1C
:106090002BF01200080E405CD8A473EF30F03DECFA
:1060A00043F0000E66EC2BF00DEC43F0000E66ECB6
:1060B0002BF01DEC46F0000E66EC2BF0FDEC45F0ED
:1060C000000E66EC2BF00DEC47F0000E66EC2BF0AA
:1060D000BDEC48F0000E66EC2BF0BDEC48F0000E75
:1060E00066EC2BF01200090E405CD8A49CEF30F057
:1060F0008DEC45F0000E66EC2BF0BDEC46F0000E8A
:1061000066EC2BF0BDEC45F0000E66EC2BF00DECD0
:1061100046F0000E66EC2BF05DEC46F0000E66ECEF
:106120002BF0BDEC48F0000E66EC2BF0BDEC48F017
:10613000000E66EC2BF012000A0E405CD8A4C5EFEE
:1061400030F0CDEC46F0000E66EC2BF02DEC46F076
:10615000000E66EC2BF08DEC46F0000E66EC2BF09A
:10616000ADEC45F0000E66EC2BF01DEC46F0000E99
:1061700066EC2BF0BDEC48F0000E66EC2BF0BDECAD
:1061800048F0000E66EC2BF012000B0E405CD8A419
:10619000A7EF31F0ADEC46F0000E66EC2BF0EDEC25
:1061A00046F0000E66EC2BF0BDEC48F0000E66ECFD
:1061B0002BF01550070B406E000E405CD8A4F6EF94
:1061C00030F08DEC46F0000E66EC2BF0EDEC46F076
:1061D000000E66EC2BF06DEC46F0000E66EC2BF03A
:1061E000ADEC42F0000E66EC2BF01200010E405CAC
:1061F000D8A410EF31F08DEC46F0000E66EC2BF0D9
:10620000EDEC46F0000E66EC2BF06DEC46F0000E67
:1062100066EC2BF0BDEC42F0000E66EC2BF01200A9
:10622000020E405CD8A42AEF31F08DEC46F0000E4F
:1062300066EC2BF0EDEC46F0000E66EC2BF06DEC0E
:1062400046F0000E66EC2BF0CDEC42F0000E66EC52
:106250002BF01200030E405CD8A444EF31F0BDECEB
:1062600046F0000E66EC2BF09DEC46F0000E66EC5E
:106270002BF09DEC45F0000E66EC2BF0BDEC48F0E9
:10628000000E66EC2BF01200040E405CD8A45EEF0A
:1062900031F08DEC46F0000E66EC2BF0EDEC46F0A4
:1062A000000E66EC2BF06DEC46F0000E66EC2BF069
:1062B000EDEC42F0000E66EC2BF01200050E405C97
:1062C000D8A478EF31F08DEC46F0000E66EC2BF0A0
:1062D000EDEC46F0000E66EC2BF06DEC46F0000E97
:1062E00066EC2BF0FDEC42F0000E66EC2BF0120099
:1062F000060E405CD8A492EF31F08DEC46F0000E13
:1063000066EC2BF0EDEC46F0000E66EC2BF06DEC3D
:1063100046F0000E66EC2BF00DEC43F0000E66EC40
:106320002BF012008DEC46F0000E66EC2BF0EDEC3D
:1063300046F0000E66EC2BF06DEC46F0000E66ECBD
:106340002BF01DEC43F0000E66EC2BF012000C0E4F
:10635000405CD8A4D0EF31F0CDEC46F0000E66ECF6
:106360002BF0BDEC45F0000E66EC2BF0BDEC45F0DB
:10637000000E66EC2BF0BDEC48F0000E66EC2BF046
:10638000BDEC48F0000E66EC2BF0BDEC48F0000EC2
:1063900066EC2BF0BDEC48F0000E66EC2BF0120022
:1063A0000D0E405CD8A4F9EF31F0FDEC45F0000E85
:1063B00066EC2BF08DEC46F0000E66EC2BF03DEC1D
:1063C00046F0000E66EC2BF0ADEC45F0000E66ECEE
:1063D0002BF01DEC46F0000E66EC2BF0BDEC48F007
:1063E000000E66EC2BF0BDEC48F0000E66EC2BF0D6
:1063F00012008DEC46F0000E66EC2BF0CDEC45F073
:10640000000E66EC2BF09DEC46F0000E66EC2BF0D7
:10641000CDEC45F0000E66EC2BF08DEC46F0000E56
:1064200066EC2BF0CDEC46F0000E66EC2BF0CDECDC
:1064300045F0000E66EC2BF0120080B039EF32F020
:10644000070E555CD8B428EF32F0552A3BEF32F0F6
:10645000556A3EB03BEF32F0000E495CD8A435EFF0
:1064600032F0080E496E36EF32F049063E803BEFBF
:1064700032F03E90556A84B657EF32F0070E545C06
:10648000D8B446EF32F0542A59EF32F0546A3EBC89
:1064900059EF32F0080E495CD8A453EF32F0000EE9
:1064A000496E54EF32F0492A3E8C59EF32F03E9C4F
:1064B000546A120080B076EF32F0070E555CD8B403
:1064C00065EF32F0552A78EF32F0556A3EB078EF3A
:1064D00032F0010E495CD8A472EF32F0080E496E1A
:1064E00073EF32F049063E8078EF32F03E90556A05
:1064F00084B694EF32F0070E545CD8B483EF32F0D8
:10650000542A96EF32F0546A3EBC96EF32F0080EF1
:10651000495CD8A490EF32F0010E496E91EF32F051
:10652000492A3E8C96EF32F03E9C546A1200080EC7
:10653000495CD8B4AEEF34F03FB4DDEF32F080B850
:10654000B2EF32F0070E575CD8B4AAEF32F0572AF8
:10655000B4EF32F0576A3EB870EF33F03F843E88B4
:10656000DDEF32F03E98576A28EC2BF04D0E34ECFC
:106570002BF0BE0E4DEC2BF0000E66EC2BF0BDECBC
:1065800048F0000E66EC2BF0BDEC48F0BDEC48F096
:10659000000E66EC2BF0BDEC48F0000E66EC2BF024
:1065A000BDEC48F0000E66EC2BF0BDEC48F0000EA0
:1065B00066EC2BF04A50406E120028EC2BF04D0E8A
:1065C00034EC2BF0BE0E4DEC2BF0000E495CD8B431
:1065D0000AEF33F0010E495CD8B40FEF33F0020E2E
:1065E000495CD8B414EF33F0030E495CD8B419EF0A
:1065F00033F0040E495CD8B41EEF33F0050E495C4D
:10660000D8B423EF33F0060E495CD8B428EF33F04A
:106610002DEF33F04BAE32EF33F052EF33F04BACA3
:1066200032EF33F052EF33F04BAA32EF33F052EF48
:1066300033F04BA832EF33F052EF33F04BA632EF8A
:1066400033F052EF33F04BA432EF33F052EF33F02C
:106650004BA232EF33F052EF33F04BA032EF33F076
:1066600052EF33F0000E66EC2BF0BDEC42F0000E62
:1066700066EC2BF0BDEC48F05DEC46F0000E66ECED
:106680002BF08DEC46F0000E66EC2BF0BDEC48F0E4
:10669000FF0E66EC2BF04DEC43F0FF0E66EC2BF09A
:1066A00070EF33F0FF0E66EC2BF05DEC43F0FF0E65
:1066B00066EC2BF0BDEC48F05DEC46F0000E66ECAD
:1066C0002BF08DEC46F0000E66EC2BF0BDEC48F0A4
:1066D000000E66EC2BF0ADEC42F0000E66EC2BF0F9
:1066E0004A50406E3FA4120080BA89EF33F0070E83
:1066F000565CD8B47FEF33F0562A8BEF33F0566AEE
:106700003EBA8BEF33F03F944A50406E4B6E3E8A58
:1067100012003E9A566A80B80DEF34F0070E575CAF
:10672000D8B496EF33F0572A0FEF34F0576A3EB8DB
:106730000FEF34F0000E495CD8B4BFEF33F0010E18
:10674000495CD8B4C8EF33F0020E495CD8B4D1EF3D
:1067500033F0030E495CD8B4DAEF33F0040E495C31
:10676000D8B4E3EF33F0050E495CD8B4ECEF33F066
:10677000060E495CD8B4F5EF33F0FEEF33F04BAEC4
:10678000C5EF33F04A8E07EF34F04A9E07EF34F03E
:106790004BACCEEF33F04A8C07EF34F04A9C07EF56
:1067A00034F04BAAD7EF33F04A8A07EF34F04A9A15
:1067B00007EF34F04BA8E0EF33F04A8807EF34F0EE
:1067C0004A9807EF34F04BA6E9EF33F04A8607EF1B
:1067D00034F04A9607EF34F04BA4F2EF33F04A84DA
:1067E00007EF34F04A9407EF34F04BA2FBEF33F09D
:1067F0004A8207EF34F04A9207EF34F04BA004EFDF
:1068000034F04A8007EF34F04A9007EF34F03F94B9
:106810004A50406E3E880FEF34F03E98576A80B081
:106820005CEF34F0070E555CD8B41AEF34F0552AFB
:106830005EEF34F0556A3EB05EEF34F0000E495C16
:10684000D8B443EF34F0010E495CD8B446EF34F0CD
:10685000020E495CD8B449EF34F0030E495CD8B459
:106860004CEF34F0040E495CD8B44FEF34F0050E11
:10687000495CD8B452EF34F0060E495CD8B455EFF9
:1068800034F058EF34F04B7E59EF34F04B7C59EF35
:1068900034F04B7A59EF34F04B7859EF34F04B76B3
:1068A00059EF34F04B7459EF34F04B7259EF34F028
:1068B0004B703E805EEF34F03E90556A84B6ABEF8D
:1068C00034F0070E545CD8B469EF34F0542AAEEFBC
:1068D00034F0546A3EBCADEF34F0000E495CD8B4DD
:1068E00092EF34F0010E495CD8B495EF34F0020E0B
:1068F000495CD8B498EF34F0030E495CD8B49BEFF0
:1069000034F0040E495CD8B49EEF34F0050E495CB7
:10691000D8B4A1EF34F0060E495CD8B4A4EF34F03B
:10692000A7EF34F04B7EA8EF34F04B7CA8EF34F0A7
:106930004B7AA8EF34F04B78A8EF34F04B76A8EF01
:1069400034F04B74A8EF34F04B72A8EF34F04B7076
:106950003E8CADEF34F03E9C546A120080B828EFB4
:1069600035F0070E575CD8B4B9EF34F0572A2AEF48
:1069700035F0576A3EB82AEF35F0000E465CD8B4C1
:10698000F0EF34F0010E465CD8B4F4EF34F0020EB0
:10699000465CD8B4F8EF34F0030E465CD8B4FCEF94
:1069A00034F0040E465CD8B400EF35F0050E465CBA
:1069B000D8B404EF35F0060E465CD8B408EF35F0D5
:1069C000070E465CD8B40CEF35F0080E465CD8B420
:1069D00010EF35F0090E465CD8B414EF35F0120014
:1069E0004A50116E16EF35F04A50126E16EF35F020
:1069F0004A50136E16EF35F04A50146E16EF35F00C
:106A00004A50156E16EF35F04A50166E16EF35F0F7
:106A10004A50176E16EF35F04A50186E16EF35F0E3
:106A20004A50196E16EF35F04A501A6E6DEC2CF084
:106A30004A50406E3E88000E465CD8B424EF35F0D4
:106A4000070E496E2AEF35F0050E496E2AEF35F034
:106A50003E98576A120028EC2BF0670E34EC2BF0AE
:106A6000BC0E4DEC2BF03FBC4AEF35F0000E66EC4F
:106A70002BF0FDEC46F0000E66EC2BF0CDEC45F073
:106A8000000E66EC2BF09DEC46F0000E66EC2BF051
:106A90005CEF35F0FF0E66EC2BF09DEC48F0FF0E3E
:106AA00066EC2BF05DEC47F0FF0E66EC2BF03DEC56
:106AB00048F0FF0E66EC2BF02BEC2BF0440E34EC80
:106AC0002BF0BC0E4DEC2BF03FBC7BEF35F0FF0EF6
:106AD00066EC2BF0EDEC47F0FF0E66EC2BF0CDEC06
:106AE00048F0FF0E66EC2BF0FDEC47F0FF0E66EC75
:106AF0002BF08DEF35F0000E66EC2BF04DEC46F0F0
:106B0000000E66EC2BF0BDEC48F0000E66EC2BF0AE
:106B10005DEC46F0000E66EC2BF080B0A6EF35F091
:106B2000070E555CD8B498EF35F0552AA8EF35F02C
:106B3000556A3EB0A8EF35F03FBCA2EF35F03F8C70
:106B4000A3EF35F03F9C3E80A8EF35F03E90556AAC
:106B500084B6C1EF35F0070E545CD8B4B3EF35F00E
:106B6000542AC3EF35F0546A3EBCC3EF35F03FBC46
:106B7000BDEF35F03F8CBEEF35F03F9C3E8CC3EF50
:106B800035F03E9C546A120080B841EF36F0070E93
:106B9000575CD8B4CFEF35F0572A43EF36F0576A39
:106BA0003EB843EF36F03FAC3BEF36F050EC2CF004
:106BB000000E475CD8B411EF36F0010E475CD8B434
:106BC00015EF36F0020E475CD8B419EF36F0030E1D
:106BD000475CD8B41DEF36F0040E475CD8B421EF03
:106BE00036F0050E475CD8B425EF36F0060E475C4C
:106BF000D8B429EF36F0070E475CD8B42DEF36F045
:106C0000080E475CD8B431EF36F0090E475CD8B4B3
:106C100035EF36F00A0E475CD8B439EF36F03BEF6B
:106C200036F0F5EC48F03BEF36F008EC49F03BEF7E
:106C300036F01BEC49F03BEF36F02EEC49F03BEF21
:106C400036F041EC49F03BEF36F054EC49F03BEFC5
:106C500036F067EC49F03BEF36F07AEC49F03BEF69
:106C600036F08DEC49F03BEF36F0A0EC49F03BEF0D
:106C700036F0B3EC49F0446A476A3F9C3E8823EF04
:106C800001F03E98576A120083A264EF36F03FB8D5
:106C900012004CB256EF36F01550380B406E180EFD
:106CA000406E1550C70B156E5EEF36F015503F0B5A
:106CB000406E1B0E406E1550C00B156E40501512E5
:106CC0006DEC2CF03F8812003F9812001550380BE5
:106CD000406E4042404240424050070B406E1550CB
:106CE000F80B156E405015121200106E000E105C5D
:106CF000D8A493EF36F005B884EF36F005BA88EFE4
:106D000036F00DEC42F01200BDEC48F0058C12009C
:106D100005BC8FEF36F0059C0DEC42F01200059C8F
:106D2000BDEC48F01200010E105CD8A49BEF36F0C9
:106D30001DEC42F01200020E105CD8A4A3EF36F056
:106D40002DEC42F01200030E105CD8A4ABEF36F02D
:106D50003DEC42F01200040E105CD8A4B3EF36F004
:106D60004DEC42F01200050E105CD8A4BBEF36F0DB
:106D70005DEC42F01200060E105CD8A4C3EF36F0B2
:106D80006DEC42F01200070E105CD8A4CBEF36F089
:106D90007DEC42F01200080E105CD8A4D3EF36F060
:106DA0008DEC42F012009DEC42F01200106E000ECD
:106DB000105CD8A4DFEF36F0ADEC42F01200010E0B
:106DC000105CD8A4E7EF36F0BDEC42F01200020EE2
:106DD000105CD8A4EFEF36F0CDEC42F01200030EB9
:106DE000105CD8A4F7EF36F0DDEC42F01200040E90
:106DF000105CD8A4FFEF36F0EDEC42F01200050E67
:106E0000105CD8A407EF37F0FDEC42F01200060E3C
:106E1000105CD8A40FEF37F00DEC43F01200070E12
:106E2000105CD8A417EF37F01DEC43F01200080EE9
:106E3000105CD8A41FEF37F02DEC43F012003DECAE
:106E400043F01200106E000E105CD8A42BEF37F048
:106E50004DEC43F01200010E105CD8A433EF37F074
:106E60005DEC43F01200020E105CD8A43BEF37F04B
:106E70006DEC43F01200030E105CD8A443EF37F022
:106E80007DEC43F01200040E105CD8A44BEF37F0F9
:106E90008DEC43F01200050E105CD8A453EF37F0D0
:106EA0009DEC43F01200060E105CD8A45BEF37F0A7
:106EB000ADEC43F01200070E105CD8A463EF37F07E
:106EC000BDEC43F01200080E105CD8A46BEF37F055
:106ED000CDEC43F01200DDEC43F01200062A0A0E5E
:106EE000065CD8A46EEF37F0066A1200062AFF0E81
:106EF000065CD8A476EF37F0066A072A640E075CB2
:106F0000D8A476EF37F0066A076A1200062AFF0E49
:106F1000065CD8A486EF37F0066A072AFF0E075CE6
:106F2000D8A486EF37F0066A076A120028EC2BF027
:106F3000400E34EC2BF0BF0E4DEC2BF0BDEC45F0C9
:106F4000000E66EC2BF08DEC45F0000E66EC2BF09D
:106F50000DEC46F0000E66EC2BF02DEC43F0000E2D
:106F600066EC2BF0EDEC42F0000E66EC2BF0BDEC85
:106F700042F0000E66EC2BF00DEC43F0BDEC48F057
:106F80008DEC46F0000E66EC2BF0CDEC45F0000EDB
:106F900066EC2BF0CDEC46F02BEC2BF0400E34ECF5
:106FA0002BF0BF0E4DEC2BF0400E66EC2BF0000EDC
:106FB00066EC2BF0BDEC42F0000E66EC2BF0400EC0
:106FC00066EC2BF0000E66EC2BF0ADEC42F0000E00
:106FD00066EC2BF0400E036E7F0E046E28EC2BF057
:106FE000035034EC2BF0BC0E4DEC2BF0010E66EC94
:106FF0002BF02BEC2BF0045034EC2BF0BC0E4DECB2
:107000002BF0010E66EC2BF0032A040676EC37F029
:10701000800E035CD8A4EEEF37F086EC37F086ECF8
:1070200037F086EC37F086EC37F086EC37F0400E20
:10703000036E7F0E046E28EC2BF0035034EC2BF023
:10704000BC0E4DEC2BF0000E66EC2BF02BEC2BF075
:10705000045034EC2BF0BC0E4DEC2BF0000E66EC23
:107060002BF0032A040676EC37F0800E035CD8A4DC
:107070001BEF38F03F8E86EC37F086EC37F086EC6D
:1070800037F086EC37F0508028EC2BF04A0E34ECC9
:107090002BF0BB0E4DEC2BF03DEC44F0000E66ECFB
:1070A0002BF0100E66EC2BF0100E66EC2BF0100E91
:1070B00066EC2BF0100E66EC2BF0100E66EC2BF04D
:1070C000000E66EC2BF0BDEC44F0000E66EC2BF0ED
:1070D000BDEC48F0000E66EC2BF02DEC44F0000EF9
:1070E00066EC2BF0BDEC44F0000E66EC2BF04DECA2
:1070F00044F0000E66EC2BF06DEC44F0000E66ECF4
:107100002BF0BDEC44F0000E66EC2BF02BEC2BF0DA
:10711000400E34EC2BF0BB0E4DEC2BF02DEC44F07C
:10712000000E66EC2BF02DEC44F0000E66EC2BF01C
:10713000FDEC44F0000E66EC2BF06DEC44F0000E1C
:1071400066EC2BF0BDEC44F0000E66EC2BF04DEC41
:1071500044F0000E66EC2BF0509028EC2BF0560E0D
:1071600034EC2BF0BC0E4DEC2BF0EDEC43F0000EAC
:1071700066EC2BF02DEC45F0000E66EC2BF01DECD0
:1071800044F0000E66EC2BF06DEC44F0000E66EC63
:107190002BF0CDEC44F0000E66EC2BF0BDEC48F08B
:1071A000000E66EC2BF09DEC44F0000E66EC2BF02C
:1071B0002BEC2BF0400E34EC2BF0BC0E4DEC2BF0F6
:1071C000EDEC43F0000E66EC2BF0FDEC43F0000E0E
:1071D00066EC2BF0CDEC44F0000E66EC2BF0FDECF1
:1071E00044F0000E66EC2BF0EDEC43F0000E66EC84
:1071F0002BF01DEC45F0000E66EC2BF0CDEC44F0CE
:10720000000E66EC2BF0FDEC44F0000E66EC2BF06B
:107210006DEC45F0000E66EC2BF0512A080E515C27
:10722000D8A43BEF38F03F9E516A86EC37F086ECED
:1072300037F086EC37F086EC37F086EC37F086ECEA
:1072400037F086EC37F086EC37F086EC37F086ECDA
:1072500037F086EC37F086EC37F086EC37F086ECCA
:1072600037F086EC37F086EC37F086EC37F086ECBA
:1072700037F086EC37F086EC37F086EC37F086ECAA
:1072800037F086EC37F086EC37F086EC37F086EC9A
:1072900037F086EC37F086EC37F086EC37F086EC8A
:1072A00037F086EC37F086EC37F086EC37F086EC7A
:1072B00037F086EC37F086EC37F086EC37F086EC6A
:1072C00037F086EC37F086EC37F086EC37F086EC5A
:1072D00037F086EC37F086EC37F086EC37F086EC4A
:1072E00037F086EC37F086EC37F086EC37F086EC3A
:1072F00037F086EC37F086EC37F086EC37F086EC2A
:1073000037F086EC37F086EC37F086EC37F086EC19
:1073100037F086EC37F086EC37F086EC37F086EC09
:1073200037F086EC37F086EC37F086EC37F086ECF9
:1073300037F086EC37F086EC37F086EC37F086ECE9
:1073400037F086EC37F086EC37F086EC37F086ECD9
:1073500037F050EC2CF086EC37F086EC37F086EC0A
:1073600037F086EC37F01200096E640E095ED8A083
:10737000BDEF39F00A2AB5EF39F0640E09260A0E7E
:10738000095ED8A0C7EF39F00B2ABFEF39F00A0E1B
:107390000926010E095ED8A0D1EF39F00C2AC9EFF9
:1073A00039F012000D6E100E0D5ED8A0DBEF39F033
:1073B0000B2AD3EF39F0100E0D26010E0D5ED8A06A
:1073C000E5EF39F00C2ADDEF39F0120005880A509C
:1073D00075EC36F0000E66EC2BF00598058A0B5024
:1073E00075EC36F0000E66EC2BF0059A0C5075EC3F
:1073F00036F0000E66EC2BF00A6A0B6A0C6A12007B
:107400000A50D6EC36F0000E66EC2BF00B50D6ECA2
:1074100036F0000E66EC2BF00C50D6EC36F0000E79
:1074200066EC2BF00A6A0B6A0C6A12000A5022EC16
:1074300037F0FF0E66EC2BF00B5022EC37F0FF0E0E
:1074400066EC2BF00C5022EC37F0FF0E66EC2BF0C4
:107450000A6A0B6A0C6A1200406E452A090E455CE6
:10746000D8B442EF3AF040BE3AEF3AF0ADEC42F019
:107470003CEF3AF0BDEC42F0000E66EC2BF04046DB
:107480002DEF3AF0456A1200406E080E455CD8B404
:1074900081EF3AF040BE66EF3AF04550495CD8B40F
:1074A0005CEF3AF0000E66EC2BF0ADEC42F0000E13
:1074B00066EC2BF07DEF3AF0FF0E66EC2BF04DEC16
:1074C00043F0FF0E66EC2BF07DEF3AF04550495C3F
:1074D000D8B475EF3AF0000E66EC2BF0BDEC42F03C
:1074E000000E66EC2BF07DEF3AF0FF0E66EC2BF011
:1074F0005DEC43F0FF0E66EC2BF0452A404645EF6D
:107500003AF0456A12007D0E4F5CD8B48AEF3AF02B
:107510004F2A12003F8A4F6A12002BEC2BF0530EB9
:1075200034EC2BF0BE0E4DEC2BF0080E495CD8A4C9
:10753000E5EF3AF0FF0E66EC2BF03DEC48F0FF0E65
:1075400066EC2BF05DEC47F0FF0E66EC2BF04DEC9B
:1075500048F0FF0E66EC2BF028EC2BF0460E34ECD6
:107560002BF0BC0E4DEC2BF0000E66EC2BF0BDECBE
:1075700048F0000E66EC2BF0BDEC48F0000E66EC17
:107580002BF0BDEC48F0000E66EC2BF0BDEC48F0A3
:10759000000E66EC2BF0BDEC48F0000E66EC2BF014
:1075A000BDEC48F0000E66EC2BF0BDEC48F0000E90
:1075B00066EC2BF0BDEC48F0000E66EC2BF0BDEC59
:1075C00048F0000E66EC2BF01200000E66EC2BF07B
:1075D0009DEC46F0000E66EC2BF0CDEC45F0000E75
:1075E00066EC2BF0ADEC46F0000E66EC2BF01200D2
:1075F0002BEC2BF0400E34EC2BF0BB0E4DEC2BF0B3
:107600001200000E66EC2BF04DEC46F0000E66EC1E
:107610002BF05DEC46F0000E66EC2BF0BDEC48F074
:10762000000E66EC2BF083EC3CF0BDEC48F0000E55
:1076300066EC2BF0BDEC48F0BDEC48F0DEEC3CF025
:107640001200FF0E66EC2BF01DEC48F0FF0E66EC0E
:107650002BF03DEC47F0FF0E66EC2BF02DEC48F0E4
:10766000FF0E66EC2BF03DEC47F0FF0E66EC2BF0C6
:10767000CDEC48F0FF0E66EC2BF09DEC3CF0DEEC20
:107680003CF01200FF0E66EC2BF03DEC47F0FF0ED5
:1076900066EC2BF03DEC47F0FF0E66EC2BF02DEC8A
:1076A00048F0FF0E66EC2BF03DEC47F0FF0E66EC69
:1076B0002BF0CDEC48F0FF0E66EC2BF09DEC3CF08F
:1076C000DEEC3CF01200FF0E66EC2BF05DEC48F0B7
:1076D000FF0E66EC2BF0EDEC47F0FF0E66EC2BF0A6
:1076E000CDEC47F0FF0E66EC2BF0FDEC47F0FF0E03
:1076F00066EC2BF03DEC47F0FF0E66EC2BF0BDEC9A
:1077000047F0FF0E66EC2BF0BDEC48F0000E66EC87
:107710002BF0BDEC48F0000E66EC2BF0BDEC48F011
:10772000000E66EC2BF0BDEC48F0000E66EC2BF082
:10773000DEEC3CF01200FF0E66EC2BF06DEC48F036
:10774000FF0E66EC2BF01DEC47F0FF0E66EC2BF005
:10775000CDEC47F0FF0E66EC2BF09DEC47F0FF0EF2
:1077600066EC2BF04DEC47F0FF0E66EC2BF09DEC39
:1077700047F0FF0E66EC2BF04DEC48F0FF0E66EC88
:107780002BF09DEC48F0FF0E66EC2BF0CDEC48F0B2
:107790005DEC47F0FF0E66EC2BF0810E66EC2BF0F3
:1077A000ED0E66EC2BF0ED0E66EC2BF0ED0E66ECBC
:1077B0002BF0F8EC3AF0930E66EC2BF0FF0E66EC33
:1077C0002BF0A7EC3CF0BDEC48F0000E66EC2BF083
:1077D0001200FF0E66EC2BF02DEC47F0FF0E66EC6E
:1077E0002BF09DEC47F0FF0E66EC2BF0CDEC48F053
:1077F000FF0E66EC2BF00DEC48F0FF0E66EC2BF064
:107800008DEC47F0FF0E66EC2BF01DEC47F0FF0E01
:1078100066EC2BF03DEC48F0FF0E66EC2BF05DECD7
:1078200047F0FF0E66EC2BF0CDEC48F05DEC47F036
:10783000FF0E66EC2BF0810E66EC2BF0ED0E66EC85
:107840002BF0ED0E66EC2BF0ED0E66EC2BF0F8EC69
:107850003AF0930E66EC2BF0FF0E66EC2BF0A7ECE3
:107860003CF0BDEC48F0000E66EC2BF01200FF0E71
:1078700066EC2BF00DEC48F0FF0E66EC2BF01DECE7
:1078800047F0FF0E66EC2BF02DEC48F0FF0E66EC97
:107890002BF09DEC47F0FF0E66EC2BF04DEC48F022
:1078A000FF0E66EC2BF09DEC48F0FF0E66EC2BF023
:1078B000CDEC48F05DEC47F0FF0E66EC2BF02DECC4
:1078C00048F0FF0E66EC2BF02DEC48F0FF0E66EC56
:1078D0002BF0C30E66EC2BF0BD0E66EC2BF0BD0E4C
:1078E00066EC2BF0BD0E66EC2BF0F8EC3AF0C30E14
:1078F00066EC2BF0FF0E66EC2BF0B1EC3CF0000ECA
:1079000066EC2BF01200CDEC45F0000E66EC2BF08F
:107910008DEC46F0000E66EC2BF08DEC46F0000E80
:1079200066EC2BF05DEC46F0000E66EC2BF08DEC77
:1079300046F0000E66EC2BF012005DEC47F0FF0EF7
:1079400066EC2BF02DEC48F0FF0E66EC2BF02DECE6
:1079500048F0FF0E66EC2BF0FDEC47F0FF0E66ECF6
:107960002BF02DEC48F0FF0E66EC2BF012009DEC96
:107970003CF0CDEC48F0FF0E66EC2BF03DEC47F010
:10798000FF0E66EC2BF0FDEC47F0FF0E66EC2BF0E3
:107990004DEC47F0FF0E66EC2BF05DEC47F0FF0E70
:1079A00066EC2BF0FF0E66EC2BF0FF0E66EC2BF076
:1079B000FF0E66EC2BF0F8EC3AF01200F8EC3AF01F
:1079C000BDEC48F0000E66EC2BF0BDEC48F0000E6C
:1079D00066EC2BF0BDEC48F0000E66EC2BF0BDEC35
:1079E00048F0000E66EC2BF0BDEC48F0000E66ECA3
:1079F0002BF01200ADEC45F0000E66EC2BF05DECC8
:107A000046F0000E66EC2BF04DEC46F0000E66ECF6
:107A10002BF0ADEC46F0000E66EC2BF08DEC46F052
:107A2000000E66EC2BF05DEC46F0000E66EC2BF0E1
:107A30002DEC46F0000E66EC2BF0BDEC48F0ADEC02
:107A400042F0000E66EC2BF0BDEC48F02BEC2BF076
:107A5000400E34EC2BF0B90E4DEC2BF0FF0E66EC23
:107A60002BF0810E66EC2BF0810E66EC2BF0000EF5
:107A700066EC2BF0ADEC42F0000E66EC2BF0ADECBA
:107A800042F0000E66EC2BF0FDEC45F0000E66ECCB
:107A90002BF0810E66EC2BF0810E66EC2BF0FF0EC6
:107AA00066EC2BF01200ADEC45F0000E66EC2BF00E
:107AB0005DEC46F0000E66EC2BF04DEC46F0000E4F
:107AC00066EC2BF0ADEC46F0000E66EC2BF08DEC86
:107AD00046F0000E66EC2BF05DEC46F0000E66EC16
:107AE0002BF02DEC46F0000E66EC2BF0BDEC48F0D0
:107AF000BDEC42F0000E66EC2BF0BDEC48F02BEC38
:107B00002BF0400E34EC2BF0B90E4DEC2BF0FF0EA9
:107B100066EC2BF0810E66EC2BF0810E66EC2BF000
:107B2000000E66EC2BF0ADEC42F0000E66EC2BF094
:107B3000BDEC42F0000E66EC2BF0FDEC45F0000EC3
:107B400066EC2BF0810E66EC2BF0810E66EC2BF0D0
:107B5000FF0E66EC2BF01200ADEC45F0000E66EC6B
:107B60002BF05DEC46F0000E66EC2BF04DEC46F091
:107B7000000E66EC2BF0ADEC46F0000E66EC2BF040
:107B80008DEC46F0000E66EC2BF05DEC46F0000E3E
:107B900066EC2BF02DEC46F0000E66EC2BF0BDEC05
:107BA00048F0CDEC42F0000E66EC2BF0BDEC48F056
:107BB0002BEC2BF0400E34EC2BF0B90E4DEC2BF0EF
:107BC000FF0E66EC2BF0810E66EC2BF0810E66EC5E
:107BD0002BF0000E66EC2BF0ADEC42F0000E66ECE4
:107BE0002BF0CDEC42F0000E66EC2BF0FDEC45F0F6
:107BF000000E66EC2BF0810E66EC2BF0810E66EC2D
:107C00002BF0FF0E66EC2BF01200ADEC45F0000EF1
:107C100066EC2BF05DEC46F0000E66EC2BF04DECC4
:107C200046F0000E66EC2BF0ADEC46F0000E66EC74
:107C30002BF08DEC46F0000E66EC2BF05DEC46F080
:107C4000000E66EC2BF02DEC46F0000E66EC2BF0EF
:107C5000BDEC48F0DDEC42F0000E66EC2BF0BDEC24
:107C600048F02BEC2BF0400E34EC2BF0B90E4DEC21
:107C70002BF0FF0E66EC2BF0810E66EC2BF0810EE4
:107C800066EC2BF0000E66EC2BF0ADEC42F0000E33
:107C900066EC2BF0DDEC42F0000E66EC2BF0FDEC18
:107CA00045F0000E66EC2BF0810E66EC2BF0810E99
:107CB00066EC2BF0FF0E66EC2BF01200ADEC45F0FD
:107CC000000E66EC2BF05DEC46F0000E66EC2BF03F
:107CD0004DEC46F0000E66EC2BF0ADEC46F0000EDD
:107CE00066EC2BF08DEC46F0000E66EC2BF05DECB4
:107CF00046F0000E66EC2BF02DEC46F0000E66EC24
:107D00002BF0BDEC48F0EDEC42F0000E66EC2BF0F1
:107D1000BDEC48F02BEC2BF0400E34EC2BF0B90E00
:107D20004DEC2BF0FF0E66EC2BF0810E66EC2BF089
:107D3000810E66EC2BF0000E66EC2BF0ADEC42F001
:107D4000000E66EC2BF0EDEC42F0000E66EC2BF032
:107D5000FDEC45F0000E66EC2BF0810E66EC2BF08E
:107D6000810E66EC2BF0FF0E66EC2BF012009DEC02
:107D700046F0000E66EC2BF0CDEC45F0000E66EC04
:107D80002BF08DEC46F0000E66EC2BF00DEC46F07F
:107D9000000E66EC2BF08DEC45F0000E66EC2BF03F
:107DA0002DEC46F0000E66EC2BF0BDEC48F08DECAF
:107DB00045F0000E66EC2BF0BDEC46F0000E66ECD4
:107DC0002BF0BDEC45F02BEC2BF0400E34EC2BF0FF
:107DD000B90E4DEC2BF0000E66EC2BF00DEC46F0DE
:107DE000000E66EC2BF05DEC46F0000E66EC2BF01E
:107DF00028EC2BF04C0E34EC2BF0BA0E4DEC2BF0A3
:107E0000BDEC45F0000E66EC2BF08DEC45F0000E5D
:107E100066EC2BF0ADEC46F0000E66EC2BF08DEC32
:107E200045F0000E66EC2BF0BDEC48F0DDEC45F0C3
:107E3000000E66EC2BF05DEC46F0000E66EC2BF0CD
:107E40008DEC46F0000E66EC2BF03DEC46F02BEC92
:107E50002BF0400E34EC2BF0BA0E4DEC2BF0000E54
:107E600066EC2BF08DEC45F0000E66EC2BF0ADECE3
:107E700046F0BDEC48F0FF0E66EC2BF0810E66EC90
:107E80002BF0810E66EC2BF0000E66EC2BF0ADECC7
:107E900042F0000E66EC2BF0FDEC42F0000E66ECBA
:107EA0002BF0FDEC45F0000E66EC2BF0810E66EC3D
:107EB0002BF0810E66EC2BF0FF0E66EC2BF012001F
:107EC0008DEC46F0000E66EC2BF0CDEC45F0000E8C
:107ED00066EC2BF0ADEC45F0000E66EC2BF0CDEC33
:107EE00045F0000E66EC2BF00DEC46F0000E66EC53
:107EF0002BF0CDEC46F0000E66EC2BF0CDEC45F00F
:107F0000000E66EC2BF08DEC46F0000E66EC2BF0CC
:107F1000BDEC48F0CDEC45F02BEC2BF0400E34ECF2
:107F20002BF0B90E4DEC2BF0000E66EC2BF08DEC27
:107F300046F0000E66EC2BF08DEC46F0000E66EC81
:107F40002BF05DEC46F0000E66EC2BF08DEC46F06D
:107F5000000E66EC2BF0BDEC48F03DEC46F0000E58
:107F600066EC2BF08DEC45F0000E66EC2BF09DECF2
:107F700046F0000E66EC2BF01DEC46F0000E66ECB1
:107F80002BF02BEC2BF0640E34EC2BF0BA0E4DECF6
:107F90002BF0FF0E66EC2BF0810E66EC2BF0810EC1
:107FA00066EC2BF0000E66EC2BF0ADEC42F0000E10
:107FB00066EC2BF00DEC43F0000E66EC2BF0FDECC4
:107FC00045F0000E66EC2BF0810E66EC2BF0810E76
:107FD00066EC2BF0FF0E66EC2BF012000DEC46F079
:107FE000000E66EC2BF04DEC46F0000E66EC2BF02C
:107FF000ADEC46F0000E66EC2BF0CDEC45F0000E3B
:1080000066EC2BF08DEC46F0000E66EC2BF08DEC60
:1080100046F0000E66EC2BF0BDEC46F0000E66EC70
:108020002BF06DEC46F0000E66EC2BF0ADEC46F05C
:10803000BDEC48F02BEC2BF0400E34EC2BF0B90EDD
:108040004DEC2BF0000E66EC2BF03DEC46F0000EF4
:1080500066EC2BF08DEC45F0000E66EC2BF09DEC01
:1080600046F0000E66EC2BF01DEC46F0BDEC48F03F
:10807000FF0E66EC2BF0810E66EC2BF0810E66ECA9
:108080002BF0000E66EC2BF0ADEC42F0000E66EC2F
:108090002BF01DEC43F0000E66EC2BF0FDEC45F0F0
:1080A000000E66EC2BF0810E66EC2BF0810E66EC78
:1080B0002BF0FF0E66EC2BF012000DEC46F0000EDC
:1080C00066EC2BF04DEC46F0000E66EC2BF0ADECC0
:1080D00046F0000E66EC2BF0CDEC45F0000E66ECA1
:1080E0002BF08DEC46F0000E66EC2BF08DEC46F09C
:1080F000000E66EC2BF0BDEC46F0000E66EC2BF0AB
:108100006DEC46F0000E66EC2BF0ADEC46F0BDECED
:1081100048F02BEC2BF0400E34EC2BF0B90E4DEC6C
:108120002BF0000E66EC2BF03DEC46F0000E66ECFA
:108130002BF05DEC46F0000E66EC2BF0BDEC45F04C
:10814000000E66EC2BF0CDEC45F0000E66EC2BF04B
:10815000BDEC48F03DEC46F0000E66EC2BF09DECDB
:1081600046F0000E66EC2BF09DEC45F0000E66EC40
:108170002BF02BEC2BF0640E34EC2BF0BA0E4DEC04
:108180002BF0FF0E66EC2BF0810E66EC2BF0810ECF
:1081900066EC2BF0000E66EC2BF0ADEC42F0000E1E
:1081A00066EC2BF02DEC43F0000E66EC2BF0FDECB2
:1081B00045F0000E66EC2BF0810E66EC2BF0810E84
:1081C00066EC2BF0FF0E66EC2BF012000DEC46F087
:1081D000000E66EC2BF04DEC46F0000E66EC2BF03A
:1081E000ADEC46F0000E66EC2BF0CDEC45F0000E49
:1081F00066EC2BF08DEC46F0000E66EC2BF08DEC6F
:1082000046F0000E66EC2BF0BDEC46F0000E66EC7E
:108210002BF06DEC46F0000E66EC2BF0ADEC46F06A
:10822000BDEC48F02BEC2BF0400E34EC2BF0B90EEB
:108230004DEC2BF0000E66EC2BF03DEC46F0000E02
:1082400066EC2BF05DEC46F0000E66EC2BF0BDEC1E
:1082500045F0000E66EC2BF0CDEC45F0000E66EC20
:108260002BF0BDEC48F02DEC46F0000E66EC2BF048
:108270009DEC46F0000E66EC2BF09DEC45F0000EF8
:1082800066EC2BF02BEC2BF0640E34EC2BF0BA0EDA
:108290004DEC2BF0FF0E66EC2BF0810E66EC2BF014
:1082A000810E66EC2BF0000E66EC2BF0ADEC42F08C
:1082B000000E66EC2BF03DEC43F0000E66EC2BF06C
:1082C000FDEC45F0000E66EC2BF0810E66EC2BF019
:1082D000810E66EC2BF0FF0E66EC2BF01200FF0E09
:1082E00066EC2BF00DEC48F0FF0E66EC2BF03DEC4D
:1082F00047F0FF0E66EC2BF03DEC47F0FF0E66EC0E
:108300002BF08DEC47F0FF0E66EC2BF01200FF0E09
:1083100066EC2BF0FDEC47F0FF0E66EC2BF03DEC2D
:1083200048F0FF0E66EC2BF0CDEC47F0FF0E66EC4C
:108330002BF09DEC47F0FF0E66EC2BF00DEC48F0B7
:10834000FF0E66EC2BF01200FF0E66EC2BF04DECEE
:1083500047F0FF0E66EC2BF05DEC47F0FF0E66EC8D
:108360002BF04DEC48F0FF0E66EC2BF03DEC47F0A7
:10837000FF0E66EC2BF01200FF0E66EC2BF03DECCE
:1083800047F0FF0E66EC2BF03DEC47F0FF0E66EC7D
:108390002BF08DEC47F0FF0E66EC2BF01200FF0E79
:1083A00066EC2BF02DEC48F0FF0E66EC2BF05DEC4C
:1083B00047F0FF0E66EC2BF02DEC48F0FF0E66EC5C
:1083C0002BF02DEC48F0FF0E66EC2BF01200FF0EA8
:1083D00066EC2BF01DEC48F0FF0E66EC2BF03DEC4C
:1083E00047F0FF0E66EC2BF08DEC47F0FF0E66ECCD
:1083F0002BF01200FF0E66EC2BF06DEC47F0FF0E39
:1084000066EC2BF03DEC47F0FF0E66EC2BF08DECAC
:1084100047F0FF0E66EC2BF012007C0E66EC2BF0A2
:10842000820E66EC2BF0820E66EC2BF0820E66EC70
:108430002BF07C0E66EC2BF01200000E66EC2BF09D
:10844000840E66EC2BF0FE0E66EC2BF0800E66ECD4
:108450002BF0000E66EC2BF01200E20E66EC2BF017
:10846000920E66EC2BF0920E66EC2BF0920E66EC00
:108470002BF08C0E66EC2BF01200440E66EC2BF009
:10848000820E66EC2BF0920E66EC2BF0920E66ECF0
:108490002BF06C0E66EC2BF01200300E66EC2BF01D
:1084A000280E66EC2BF0240E66EC2BF0FE0E66EC2C
:1084B0002BF0200E66EC2BF012004E0E66EC2BF02B
:1084C0008A0E66EC2BF08A0E66EC2BF08A0E66ECB8
:1084D0002BF0720E66EC2BF012007C0E66EC2BF08B
:1084E000920E66EC2BF0920E66EC2BF0920E66EC80
:1084F0002BF0640E66EC2BF01200060E66EC2BF0EF
:10850000020E66EC2BF0C20E66EC2BF0320E66EC1F
:108510002BF00E0E66EC2BF012006C0E66EC2BF0BE
:10852000920E66EC2BF0920E66EC2BF0920E66EC3F
:108530002BF06C0E66EC2BF012004C0E66EC2BF060
:10854000920E66EC2BF0920E66EC2BF0920E66EC1F
:108550002BF07C0E66EC2BF012003C0E66EC2BF040
:10856000420E66EC2BF0420E66EC2BF0420E66ECEF
:108570002BF03C0E66EC2BF01200000E66EC2BF09C
:10858000440E66EC2BF07E0E66EC2BF0400E66EC93
:108590002BF0000E66EC2BF01200720E66EC2BF046
:1085A0004A0E66EC2BF04A0E66EC2BF04A0E66EC97
:1085B0002BF0440E66EC2BF01200220E66EC2BF032
:1085C0004A0E66EC2BF04A0E66EC2BF04A0E66EC77
:1085D0002BF0340E66EC2BF01200300E66EC2BF014
:1085E000280E66EC2BF0240E66EC2BF07E0E66EC6B
:1085F0002BF0200E66EC2BF012002E0E66EC2BF00A
:108600004A0E66EC2BF04A0E66EC2BF04A0E66EC36
:108610002BF0320E66EC2BF012003C0E66EC2BF0C9
:108620004A0E66EC2BF04A0E66EC2BF04A0E66EC16
:108630002BF0300E66EC2BF01200060E66EC2BF0E1
:10864000020E66EC2BF0620E66EC2BF0120E66EC5E
:108650002BF00E0E66EC2BF01200340E66EC2BF0B5
:108660004A0E66EC2BF04A0E66EC2BF04A0E66ECD6
:108670002BF0340E66EC2BF012000C0E66EC2BF097
:10868000520E66EC2BF0520E66EC2BF0520E66EC9E
:108690002BF03C0E66EC2BF01200C30E66EC2BF0B8
:1086A000BD0E66EC2BF0BD0E66EC2BF0BD0E66EC3D
:1086B0002BF0C30E66EC2BF01200FF0E66EC2BF0D5
:1086C000BB0E66EC2BF0810E66EC2BF0BF0E66EC59
:1086D0002BF0FF0E66EC2BF012008D0E66EC2BF0EB
:1086E000B50E66EC2BF0B50E66EC2BF0B50E66EC15
:1086F0002BF0BB0E66EC2BF01200DD0E66EC2BF0BF
:10870000B50E66EC2BF0B50E66EC2BF0B50E66ECF4
:108710002BF0CB0E66EC2BF01200CF0E66EC2BF09C
:10872000D70E66EC2BF0DB0E66EC2BF0810E66ECC0
:108730002BF0DF0E66EC2BF01200D10E66EC2BF066
:10874000B50E66EC2BF0B50E66EC2BF0B50E66ECB4
:108750002BF0CD0E66EC2BF01200C30E66EC2BF066
:10876000B50E66EC2BF0B50E66EC2BF0B50E66EC94
:108770002BF0CF0E66EC2BF01200F90E66EC2BF00E
:10878000FD0E66EC2BF09D0E66EC2BF0ED0E66EC0C
:108790002BF0F10E66EC2BF01200CB0E66EC2BF0FA
:1087A000B50E66EC2BF0B50E66EC2BF0B50E66EC54
:1087B0002BF0CB0E66EC2BF01200F30E66EC2BF0D8
:1087C000AD0E66EC2BF0AD0E66EC2BF0AD0E66EC4C
:1087D0002BF0C30E66EC2BF01200F80E66EC2BF0BB
:1087E000240E66EC2BF0220E66EC2BF0240E66ECC9
:1087F0002BF0F80E66EC2BF01200FE0E66EC2BF060
:10880000920E66EC2BF0920E66EC2BF0920E66EC5C
:108810002BF06C0E66EC2BF012007C0E66EC2BF04D
:10882000820E66EC2BF0820E66EC2BF0820E66EC6C
:108830002BF0440E66EC2BF01200FE0E66EC2BF0D3
:10884000820E66EC2BF0820E66EC2BF0820E66EC4C
:108850002BF07C0E66EC2BF01200FE0E66EC2BF07B
:10886000920E66EC2BF0920E66EC2BF0920E66ECFC
:108870002BF0820E66EC2BF01200FE0E66EC2BF055
:10888000120E66EC2BF0120E66EC2BF0120E66EC5C
:108890002BF0020E66EC2BF012007C0E66EC2BF037
:1088A000820E66EC2BF0820E66EC2BF0920E66ECDC
:1088B0002BF0740E66EC2BF01200FE0E66EC2BF023
:1088C000100E66EC2BF0100E66EC2BF0100E66EC22
:1088D0002BF0FE0E66EC2BF01200000E66EC2BF077
:1088E000820E66EC2BF0FE0E66EC2BF0820E66EC30
:1088F0002BF0000E66EC2BF01200600E66EC2BF0F5
:10890000800E66EC2BF0800E66EC2BF0800E66EC91
:108910002BF07E0E66EC2BF01200FE0E66EC2BF0B8
:10892000100E66EC2BF0280E66EC2BF0440E66EC75
:108930002BF0820E66EC2BF01200FE0E66EC2BF094
:10894000800E66EC2BF0800E66EC2BF0800E66EC51
:108950002BF0800E66EC2BF01200FE0E66EC2BF076
:10896000040E66EC2BF0080E66EC2BF0040E66ECA1
:108970002BF0FE0E66EC2BF01200FE0E66EC2BF0D8
:10898000080E66EC2BF0100E66EC2BF0200E66EC59
:108990002BF0FE0E66EC2BF012007C0E66EC2BF03A
:1089A000820E66EC2BF0820E66EC2BF0820E66ECEB
:1089B0002BF07C0E66EC2BF01200FE0E66EC2BF01A
:1089C000120E66EC2BF0120E66EC2BF0120E66EC1B
:1089D0002BF00C0E66EC2BF012007C0E66EC2BF0EC
:1089E000820E66EC2BF0A20E66EC2BF0420E66ECCB
:1089F0002BF0BC0E66EC2BF01200FE0E66EC2BF09A
:108A0000120E66EC2BF0120E66EC2BF0120E66ECDA
:108A10002BF0EC0E66EC2BF012004C0E66EC2BF0FB
:108A2000920E66EC2BF0920E66EC2BF0920E66EC3A
:108A30002BF0640E66EC2BF01200020E66EC2BF0AD
:108A4000020E66EC2BF0FE0E66EC2BF0020E66ECCE
:108A50002BF0020E66EC2BF012007E0E66EC2BF073
:108A6000800E66EC2BF0800E66EC2BF0800E66EC30
:108A70002BF07E0E66EC2BF012000E0E66EC2BF047
:108A8000300E66EC2BF0C00E66EC2BF0300E66EC70
:108A90002BF00E0E66EC2BF012001E0E66EC2BF087
:108AA000E00E66EC2BF0180E66EC2BF0E00E66EC98
:108AB0002BF01E0E66EC2BF01200C60E66EC2BF0AF
:108AC000280E66EC2BF0100E66EC2BF0280E66ECF0
:108AD0002BF0C60E66EC2BF012000E0E66EC2BF09F
:108AE000100E66EC2BF0E00E66EC2BF0100E66EC30
:108AF0002BF00E0E66EC2BF01200C20E66EC2BF083
:108B0000A20E66EC2BF0920E66EC2BF08A0E66EC51
:108B10002BF0860E66EC2BF01200780E66EC2BF034
:108B2000140E66EC2BF0120E66EC2BF0140E66ECB5
:108B30002BF0780E66EC2BF012007E0E66EC2BF01C
:108B40004A0E66EC2BF04A0E66EC2BF04A0E66ECF1
:108B50002BF0340E66EC2BF012003C0E66EC2BF082
:108B6000420E66EC2BF0420E66EC2BF0420E66ECE9
:108B70002BF0240E66EC2BF012007E0E66EC2BF030
:108B8000420E66EC2BF0420E66EC2BF0420E66ECC9
:108B90002BF03C0E66EC2BF012007E0E66EC2BF0F8
:108BA0004A0E66EC2BF04A0E66EC2BF04A0E66EC91
:108BB0002BF0420E66EC2BF012007E0E66EC2BF0D2
:108BC0000A0E66EC2BF00A0E66EC2BF00A0E66EC31
:108BD0002BF0020E66EC2BF012003C0E66EC2BF034
:108BE000420E66EC2BF0420E66EC2BF0520E66EC59
:108BF0002BF0340E66EC2BF012007E0E66EC2BF0A0
:108C0000080E66EC2BF0080E66EC2BF0080E66ECF6
:108C10002BF07E0E66EC2BF01200000E66EC2BF0B3
:108C2000420E66EC2BF07E0E66EC2BF0420E66ECEC
:108C30002BF0000E66EC2BF012007E0E66EC2BF093
:108C4000100E66EC2BF0080E66EC2BF0140E66ECA2
:108C50002BF0620E66EC2BF012007E0E66EC2BF011
:108C6000400E66EC2BF0400E66EC2BF0400E66ECEE
:108C70002BF0400E66EC2BF012007E0E66EC2BF013
:108C8000040E66EC2BF0080E66EC2BF0040E66EC7E
:108C90002BF07E0E66EC2BF012007E0E66EC2BF0B5
:108CA000040E66EC2BF0180E66EC2BF0200E66EC32
:108CB0002BF07E0E66EC2BF012003C0E66EC2BF0D7
:108CC000420E66EC2BF0420E66EC2BF0420E66EC88
:108CD0002BF03C0E66EC2BF012007E0E66EC2BF0B7
:108CE000120E66EC2BF0120E66EC2BF0120E66ECF8
:108CF0002BF00C0E66EC2BF012003C0E66EC2BF009
:108D0000420E66EC2BF0520E66EC2BF0220E66EC57
:108D10002BF05C0E66EC2BF012007E0E66EC2BF056
:108D2000120E66EC2BF0120E66EC2BF0120E66ECB7
:108D30002BF06C0E66EC2BF01200440E66EC2BF060
:108D40004A0E66EC2BF04A0E66EC2BF04A0E66ECEF
:108D50002BF0320E66EC2BF01200020E66EC2BF0BC
:108D6000020E66EC2BF07E0E66EC2BF0020E66EC2B
:108D70002BF0020E66EC2BF012003E0E66EC2BF090
:108D8000400E66EC2BF0400E66EC2BF0400E66ECCD
:108D90002BF03E0E66EC2BF01200060E66EC2BF06C
:108DA000180E66EC2BF0600E66EC2BF0180E66ECDD
:108DB0002BF0060E66EC2BF012007E0E66EC2BF00C
:108DC000200E66EC2BF0100E66EC2BF0200E66ECFD
:108DD0002BF07E0E66EC2BF01200460E66EC2BF0AC
:108DE000280E66EC2BF0100E66EC2BF0280E66ECCD
:108DF0002BF0460E66EC2BF01200060E66EC2BF004
:108E0000080E66EC2BF0700E66EC2BF0080E66EC8C
:108E10002BF0060E66EC2BF01200440E66EC2BF0E5
:108E2000640E66EC2BF0540E66EC2BF04C0E66ECE8
:108E30002BF0440E66EC2BF01200870E66EC2BF044
:108E4000EB0E66EC2BF0ED0E66EC2BF0EB0E66EC09
:108E50002BF0870E66EC2BF01200810E66EC2BF0E7
:108E6000B50E66EC2BF0B50E66EC2BF0B50E66EC8D
:108E70002BF0CB0E66EC2BF01200C30E66EC2BF041
:108E8000BD0E66EC2BF0BD0E66EC2BF0BD0E66EC55
:108E90002BF0DB0E66EC2BF01200810E66EC2BF053
:108EA000BD0E66EC2BF0BD0E66EC2BF0BD0E66EC35
:108EB0002BF0C30E66EC2BF01200810E66EC2BF04B
:108EC000B50E66EC2BF0B50E66EC2BF0B50E66EC2D
:108ED0002BF0BD0E66EC2BF01200810E66EC2BF031
:108EE000F50E66EC2BF0F50E66EC2BF0F50E66EC4D
:108EF0002BF0FD0E66EC2BF01200C30E66EC2BF08F
:108F0000BD0E66EC2BF0BD0E66EC2BF0AD0E66ECE4
:108F10002BF0CB0E66EC2BF01200810E66EC2BF0E2
:108F2000F70E66EC2BF0F70E66EC2BF0F70E66EC06
:108F30002BF0810E66EC2BF01200FF0E66EC2BF08E
:108F4000BD0E66EC2BF0810E66EC2BF0BD0E66ECD0
:108F50002BF0FF0E66EC2BF01200CF0E66EC2BF020
:108F6000BF0E66EC2BF0BF0E66EC2BF0BF0E66EC6E
:108F70002BF0C10E66EC2BF01200810E66EC2BF08C
:108F8000EF0E66EC2BF0F70E66EC2BF0EB0E66ECBA
:108F90002BF09D0E66EC2BF01200810E66EC2BF090
:108FA000BF0E66EC2BF0BF0E66EC2BF0BF0E66EC2E
:108FB0002BF0BF0E66EC2BF01200810E66EC2BF04E
:108FC000FB0E66EC2BF0F70E66EC2BF0FB0E66EC5E
:108FD0002BF0810E66EC2BF01200810E66EC2BF06C
:108FE000FB0E66EC2BF0E70E66EC2BF0DF0E66EC6A
:108FF0002BF0810E66EC2BF01200C30E66EC2BF00A
:10900000BD0E66EC2BF0BD0E66EC2BF0BD0E66ECD3
:109010002BF0C30E66EC2BF01200810E66EC2BF0E9
:10902000ED0E66EC2BF0ED0E66EC2BF0ED0E66EC23
:109030002BF0F30E66EC2BF01200C30E66EC2BF057
:10904000BD0E66EC2BF0AD0E66EC2BF0DD0E66EC83
:109050002BF0A30E66EC2BF01200810E66EC2BF0C9
:10906000ED0E66EC2BF0ED0E66EC2BF0ED0E66ECE3
:109070002BF0930E66EC2BF01200BB0E66EC2BF07F
:10908000B50E66EC2BF0B50E66EC2BF0B50E66EC6B
:109090002BF0CD0E66EC2BF01200FD0E66EC2BF0E3
:1090A000FD0E66EC2BF0810E66EC2BF0FD0E66ECEF
:1090B0002BF0FD0E66EC2BF01200C10E66EC2BF0CF
:1090C000BF0E66EC2BF0BF0E66EC2BF0BF0E66EC0D
:1090D0002BF0C10E66EC2BF01200F90E66EC2BF0B3
:1090E000E70E66EC2BF09F0E66EC2BF0E70E66ECBD
:1090F0002BF0F90E66EC2BF01200810E66EC2BF0D3
:10910000DF0E66EC2BF0EF0E66EC2BF0DF0E66EC5C
:109110002BF0810E66EC2BF01200B90E66EC2BF0F2
:10912000D70E66EC2BF0EF0E66EC2BF0D70E66EC4C
:109130002BF0B90E66EC2BF01200F90E66EC2BF05A
:10914000F70E66EC2BF08F0E66EC2BF0F70E66EC4C
:109150002BF0F90E66EC2BF01200000E66EC2BF0F3
:10916000000E66EC2BF0040E66EC2BF00A0E66EC9B
:109170002BF0040E66EC2BF01200000E66EC2BF0C8
:10918000000E66EC2BF0000E66EC2BF0000E66EC89
:109190002BF0000E66EC2BF01200FF0E66EC2BF0AD
:1091A000FF0E66EC2BF0FF0E66EC2BF0FF0E66EC6C
:1091B0002BF0FF0E66EC2BF01200280E66EC2BF065
:1091C0001200FE0E66EC2BF0FE0E66EC2BF0000E8D
:1091D00066EC2BF01200000E66EC2BF0000E66EC35
:1091E0002BF0000E66EC2BF01200000EAA6E000EA3
:1091F000A96E1150A86EA69EA69CA684550EA76EB9
:10920000AA0EA76EA682A6B203EF49F0A69412009A
:10921000000EAA6E010EA96E1250A86EA69EA69C04
:10922000A684550EA76EAA0EA76EA682A6B216EF4A
:1092300049F0A6941200000EAA6E020EA96E1350F9
:10924000A86EA69EA69CA684550EA76EAA0EA76E13
:10925000A682A6B229EF49F0A6941200000EAA6ECB
:10926000030EA96E1450A86EA69EA69CA684550E49
:10927000A76EAA0EA76EA682A6B23CEF49F0A694EE
:109280001200000EAA6E040EA96E1550A86EA69EBE
:10929000A69CA684550EA76EAA0EA76EA682A6B29D
:1092A0004FEF49F0A6941200000EAA6E050EA96EAB
:1092B0001650A86EA69EA69CA684550EA76EAA0E52
:1092C000A76EA682A6B262EF49F0A6941200000E25
:1092D000AA6E060EA96E1750A86EA69EA69CA6841E
:1092E000550EA76EAA0EA76EA682A6B275EF49F01C
:1092F000A6941200000EAA6E070EA96E1850A86E52
:10930000A69EA69CA684550EA76EAA0EA76EA68240
:10931000A6B288EF49F0A6941200000EAA6E080EBD
:10932000A96E1950A86EA69EA69CA684550EA76E7F
:10933000AA0EA76EA682A6B29BEF49F0A6941200D1
:10934000000EAA6E090EA96E1A50A86EA69EA69CC3
:10935000A684550EA76EAA0EA76EA682A6B2AEEF81
:1093600049F0A6941200000EAA6E0A0EA96E4C9E39
:109370004C50A86EA69EA69CA684550EA76EAA0E5B
:0E938000A76EA682A6B2C2EF49F0A694120014
:020000040030CA
:03000100331800B1
:02000500358044
:060008000FC00FE00F40E5
:0200000400F00A
:0C00000008044BBB9B887F7F00000000C1
:00000001FF
